:020000041100E9
:10300000002370B5284C0120636101F02DFA4020A7
:103010000223FE21254A207401F0ACFA002833D1A6
:103020000223FF21224A207C01F0A4FA00282BD1A0
:10303000204BA2899A4224D1E3891F4A93420CD1A2
:103040001E4B63611E4B2268002A03D1002B01D066
:1030500023CB23C401F07CFA70BD1A4A934201D0FD
:103060000023F0E7184B194A1B68934205D9C02288
:103070000421207C920001F0F7FA104B6361144B9D
:10308000E1E700232374EBE7CC223820AC21920146
:10309000207401F0E9FA0028F3D10E4B63610E4B66
:1030A000E3810E4BCFE7C0468863FF1F9463FF1F89
:1030B0009663FF1F5959000083050000C9420011A3
:1030C0007CBE001182150000AC63FF1F8713000057
:1030D00088BE001165430011AAAAFFFF70BE00114F
:1030E000F7B5164B0192C318021D002000938823E8
:1030F0005B05D3181B685C1C1AD09CB2402C18D8F6
:103100008D781E0CAC466746CD782D023D43AE420D
:1031100006D1019800280ED110000C70240A4C70C2
:1031200003249BB20733A343D218009B9A42DED3F9
:10313000FEBD4432F9E71000FAE7C046FC0F00007C
:10314000802213B503000324019189B25201073193
:103150009B18A14304305A1A88235B05C3181B68C7
:10316000591C03D190429241104016BD99B240299A
:1031700007D80B000733A343C0189042ECD30020BC
:10318000F3E74430F9E7134B134A1B68126810B594
:10319000FA24934201D81A00F824104BE4021B6869
:1031A0009A4210D813000E4A12689A420ED3013385
:1031B00007D1F823DB029C4203D10A49054808F0F5
:1031C000FBFC200010BDFC24E402ECE7FE24E4023A
:1031D000F7E7C04600C0071100D0071100E0071153
:1031E00000F00711FFFFFF7FF0B59BB015000490C2
:1031F0000391402A00D9A0E006AB59801A80FFF75E
:10320000C2FF0400042816D9002206A9FFF768FFB0
:10321000052810D906AB1B88AB420CD1002D07D076
:10322000514B2A000499C01808F03EFD002802D135
:1032300001201BB0F0BD06AB1D8020000699FFF7F2
:103240007FFF041E7BD1069B0793FFF79CFF802323
:103250005B01C618802307001B039E4201D3F8269A
:10326000F60288235B05F31801931B68013302D033
:10327000019808F019FB3D49019808F09DFC3B1DA1
:103280000293331D05938822029B52059B181B68ED
:1032900008935A1C3CD044219AB20091402A04D889
:1032A0000320D11D814389B2009103991B0C8B42ED
:1032B00024D0402A22D80122300008A9FFF710FFAD
:1032C000021E1BD1380008A9FFF70AFF04000428DA
:1032D00031D9009A059B9B1880225201B218934263
:1032E00040D288235B05C118009A09A808F014FC95
:1032F0001D4B009A09A9F01808F0FEFA009A029BEB
:103300009446634402931A4B029AFB189A42BAD32A
:1033100088235B05FC1821680198013908F04CFCF2
:10332000200008F0C1FA039A07AB5A8030000799D1
:10333000FFF706FF0400002C03D1002079E70428E2
:10334000FBD988235B05E018069908F035FC0323B8
:10335000EA1C9A4300D16BE7034B0499E01808F08C
:10336000CBFA65E70424ECE704000011FFFFFF7FC0
:10337000F80F0000F7B505001400402A21D80027F7
:1033800001AE71803780FFF7FEFE042816D93A009F
:103390003100FFF7A5FE042810D93688BC420BD0B7
:1033A000BD4209D0221CB44200D9321C064B92B255
:1033B000C118280008F0B0FB30B2FEBDC04300B217
:1033C000FBE703204042F8E70400001137B5042270
:1033D00004000D0001A81649FFF7CCFF02000428E5
:1033E0000BD1019BA34208D3AB4204D0104901A8E2
:1033F0000195FFF7F9FE01203EBD0E4C2368200029
:10340000019308F051FA019920000139019108F067
:10341000D3FB80235B01E418074B9C42EED10422CE
:10342000034901A80195FFF7DFFE0020E4E7C0464D
:103430005555000000C007110000081130B589B0D3
:1034400008F012FA10226946254808F0B5F9254B14
:10345000009A9A420ED1019B029A0F2B33D8002179
:1034600001240698013B08D2002900D00292029B59
:10347000013331D10023029325E0551CF2D1020023
:103480002100EFE710341022200004A908F094F97D
:10349000029B013301D1069B0293882304995B05AB
:1034A000C918059B06981A03120B049105928142D4
:1034B00003D02B4201D108F02FFB019B013B01936C
:1034C000019B002BDED1029B002B03D004930498B8
:1034D0004168084709B030BDE025014C2D03EFE7F6
:1034E0000000011150485936F7B50F490F4B0A68D3
:1034F00004001A4084235B0013430B60030003277E
:103500001033019300252E00112008F0E5FA084B36
:103510001B683B40AB4002351E43202DF4D1019B7C
:1035200040C4A342EED1F7BD5CF0004000FEFEFFB8
:1035300064F00040802270B5AD4CAE4BD20000214B
:1035400020001C6008F088FB2300AB4A88331A6017
:10355000AA4B1A786E23002A00D01133E3620A23A3
:103560002365A74B1878A74BA0630138E361C3B26A
:10357000032B01D810232362A34B37226361C82396
:10358000DB00A36123008C331A60082336210F3A35
:10359000E518E16323646264E9670439251DE9677E
:1035A00025003B26BC352E602500C0352B6025004C
:1035B000C4352A6025000636CC352E602500083E2D
:1035C000C8352E602500D03529602100D4310B602C
:1035D0002100D8310A6021000225E0310D6025006C
:1035E0004221DC35296025001B3EE4352E60250094
:1035F000E8352B602500EC352A6022000525F432E1
:1036000015602200F03211602200183190321160F2
:1036100022009432136023003C2298331A60AF23B7
:10362000DB002360794B2363032805D808F0A4FA54
:10363000330235371523636096232100FA225B009D
:10364000A360E360C8332361714BFC319200A36433
:103650000A6062626F4A704DA2627322E2656D3A3F
:103660006265A2650232E5644A60022161669621C4
:103670008900A166626709210022E166A2676749A5
:10368000674A684E2167E2673560032811D808F061
:1036900073FA96089EA61023CDE70E23CBE70C23E2
:1036A000C9E720001A259C30056020000735A030AE
:1036B00005602000A83003602300FA20F833800062
:1036C000186023006420A433186023005F38AC33F3
:1036D000186023000338B03318602300C630B433B9
:1036E000186023000020B833186023003825FC330D
:1036F0009D604D4D5A665D644C4D9A64DD61962522
:10370000AD001D624A4D9A675D62F53DFF3D9D62C9
:103710001E25484ADD6618675867D9651966DA6755
:10372000BE23C021444A5B00E250444B4900635031
:1037300004316250C4225200A350FA23E4205B00FB
:103740000432A3500432A3503D493E4A3E4BD1605F
:103750003E49800019503E49E938FF3819503D492B
:10376000043019503C491038D1613C4911633C493F
:1037700051633C4911603C49195019003B48F831EC
:1037800008603B49D16582213A4A89005A501A00A3
:1037900039490832D1671A003849B432116088219A
:1037A000374A89005A501A00364988321160364A21
:1037B000DA6408F0F9F8012008F0CEFA70BD2000B4
:1037C00014259C30056020000435A03070E72000EF
:1037D00010259C30056020000335A03068E72000EC
:1037E0000E259C30056020000235A03060E7C04601
:1037F0000004FF1F6466FF1F5071FF1F1C46FF1F60
:103800004A0AFF1F3A07000080C3C9019A0200005C
:1038100050C300006A180000280A0000204E000073
:1038200088130000F009FF1F00400011681000001D
:10383000C4090000DC05000040420F001027000012
:10384000FD1BFF1FFC00FF1F0000FF1F252FFF1F98
:103850004D32FF1FE530FF1FD91FFF1FF51FFF1F50
:10386000A121FF1F491FFF1FC528FF1F8D2CFF1F10
:10387000D918FF1FD127FF1F3925FF1F4525FF1F1F
:10388000491EFF1F011FFF1FC11DFF1FF7B50B0CB6
:10389000FF270122009300233C001E001D009446D8
:1038A000019089B262469A401000084018413618CB
:1038B000B6B2FF2F02D1012E00D19FB20098024074
:1038C0001A41AD18ADB2FF2C02D1012D00D19CB22E
:1038D0000133102BE6D10320012E07D1012D04D195
:1038E000019B2401E4191C700138FEBD102EFCD18F
:1038F0000238102DF9D00230F7E710B5064C2378C6
:10390000002B07D10548FFF7EFFD0548FFF7ECFD59
:103910000123237010BDC0462466FF1F3866FF1FB9
:103920002866FF1FF0B58BB00D0001230190102910
:1039300036D8FFF7E2FF00231A001B48C15C0133B1
:103940005218102BFAD1023B002A29D0174B184CE1
:103950001F68002306A9E25C1600FA5C56405E541C
:103960000133102BF7D102AA07F0D6FE2A0002A9D4
:10397000019808F081F908F02FF923681B182360DB
:1039800008F02AF963681B18636008F025F9A3683A
:103990001B18A36008F020F9E3681B18E3600023FC
:1039A00018000BB0F0BDC0463866FF1FBC44FF1FB7
:1039B0002866FF1F0223F0B501245D4D5D4E2B707C
:1039C0005D4B91B01C705D4F039333680820BB7052
:1039D00006F05EFC0023984205D0BA78552A02D042
:1039E000332A00D098E03360002006F0D1FE08F0C2
:1039F000BBF9FFF79FFD08F09FF81F22012400216B
:103A00004F4B10AE1A704F4B1C704F4B19704F4BF1
:103A100019689143163A0A431A6060221968914363
:103A2000403A0A431A6007F09FFF08F005F8C120EA
:103A3000FF21474B80001A588A431A50C522920032
:103A400098588843BF3901439950985841490840D4
:103A50008021C9010143802099509958C00509026D
:103A6000090A0143995080213B48490107F0CCFFE6
:103A700003232200394901940093394808F034F8AF
:103A80002C22384905A808F047F805AC6178207861
:103A9000023406F01DFCA642F8D10121002006F0F8
:103AA0002BFD314B314A196803201140A022D2026C
:103AB0000A431A608022196892040A431A6019683E
:103AC0002B4A1140802292030A431A60294B2A4A4A
:103AD000934200D8012007F0BFFF08F02DF907F04E
:103AE0005BFF287807F078FF039B1878C0B208F0D6
:103AF000D3F807F0F1FD2149042007F00DFF06F08F
:103B000013FE00F0AFF800F009FE00F097FE00F0A1
:103B100019FA002011B0F0BD00932100174A0420CB
:103B200008F0D2F88023DB059C62FFF787FC5BE797
:103B30004A0AFF1F34F000401C46FF1FB863FF1FF6
:103B4000480AFF1F490AFF1F680AFF1FBCF0004018
:103B500000E100E0FF00FFFF2046FF1FA458FF1F09
:103B60002056FF1F98BD001114F00040FF7FF8FFA2
:103B7000FFFF9FFF5071FF1F0080FF1F3B000108E8
:103B800070B500252849294A29484D6308CA1B05F4
:103B90001B0DED188242F9D10022264B8B63264B78
:103BA00008211A628022254B9205DA67244BDA68D5
:103BB0008A43DA60234A1278012A03D09A6822499C
:103BC0000A409A600121EE242048E40002686C4318
:103BD0008A430260DA6811208A43DA6008F044F808
:103BE000112007F039FE112007F04EFF184A200C73
:103BF0000400642390420AD8FA220023D2009042A3
:103C000005D9144B0A21C01807F04EFFC3B2124A5F
:103C10001372124BD4801B78002B04D1104B10214F
:103C2000187807F071FF70BD000005408805054059
:103C300000060540FF01000000F0004004E100E044
:103C40003CF000404A0AFF1FFFDFFFFF0038004042
:103C5000B70B000030F8FFFFA063FF1FDC65FF1FFC
:103C6000D863FF1F002210B51100112007F0CCFF10
:103C700010BD0000F8B5002301250826394F3A4C45
:103C80003B62E3681120AB43E360E368B343E36066
:103C900007F0E2FD112007F0E7FF112007F01CFEFE
:103CA0004023226829001343236080236268DB02DB
:103CB000134380226360A36807201343A360A368B3
:103CC0002A4A1340A3608023A2689B011343102259
:103CD000A360236C93432364236C2B4323648023CE
:103CE0005B003B62226B224B1A402263626B1A40DC
:103CF0006263A26B1A40A263E26B1340E3631D4A46
:103D0000E3681340E36006F0C9FB2900072006F0D2
:103D1000F3FB8021184A1120536C0B43536407F0C6
:103D200003FFFD21154B164A89005A508023C720F6
:103D3000626B5B0313436363E36880003343E360B8
:103D4000E368104A1D43104BE5601958114080226A
:103D500012020A431A50802292051A600B4B5E63CE
:103D6000F8BDC04600F000403CF00040FFFFDFFF20
:103D7000EFFFEFFFFFFF7FFF003800400000FF1F55
:103D8000813B0011FF00FFFF00E100E00000054063
:103D900030B503A804880B20002C0ED14968074DCC
:103DA00008784978090201430A20A94205D1012176
:103DB00020001980024B1B7A137030BD192A0000B5
:103DC000A063FF1FF7B5150008AA16884A680F4FB1
:103DD00014785278120222430A24BA4214D10122E2
:103DE000DBB2019200962A0007F0EEFB041E0BD115
:103DF000074B1B68002B07D068782A780002104315
:103E000042425041013098472000FEBD0229000087
:103E10002463FF1F30B5012503790400BFB02B4296
:103E200012D00A49408806F03BFF28420CD06A466F
:103E3000074B69465B8D55801380064B60881B7A63
:103E40001371002204F00CF83FB030BD1C63FF1F5B
:103E50006042FF1FA063FF1F10B50549054806F02B
:103E6000D5FE0421044A054806F092FE10BDC04666
:103E70001C63FF1FFFFF0000C4BD00116042FF1F55
:103E800010B5024804F06EFE10BDC046153E00118C
:103E9000062310B5837010330371443B43712A33FA
:103EA00083714433C37100230222012103720E4B3C
:103EB000027041701C8881724472197A0273C17257
:103EC0009A784273DA7882730322C2731A79027481
:103ED0005A7942740C2282749A79C274DB79037520
:103EE0001123C370152010BDA063FF1F10B514204F
:103EF00007F0A2FC124B14220021186007F0ACFE60
:103F0000002007F091FE012007F09EFC022007F040
:103F10005BFE032004F0CAF8042006F0DFF8052059
:103F200003F008FB062003F0D5FF072001F098F905
:103F3000082006F00DFE092000F086FF10BDC046E7
:103F40002863FF1F10B507F0CFFB012007F054FDD9
:103F500007F0EAFE002010BD094B10B5040098429E
:103F600005D0012904D12000064906F04FFE10BDFE
:103F70000229FCD1013904F0B3FD0028F3D0F6E7A3
:103F8000FEFF00004E63FF1F30B5012503790400DA
:103F9000BFB02B4218D00D49408806F081FE284260
:103FA00012D06A460A4B0B491B8813800B2353809F
:103FB000283313716B460A22581D07F0ADFD00220D
:103FC0006946608803F04CFF3FB030BD4E63FF1F71
:103FD000FE42FF1FA063FF1F70B50D7A100004AAF8
:103FE0002C00168810221440154220D1002E20D11A
:103FF0000A78022A18D14A68517815780E4A0902BF
:104000002943914205D00D4A914209D01C800A24CF
:1040100004E014220A491A8007F07EFD200070BDDA
:104020000C2208491A80F7E71C800124F6E70824CF
:10403000F4E70B24F2E7C046F3FF0000F4FF0000B2
:10404000A044FF1FA0BE001110B504000749084896
:1040500006F0DCFD074804F0C5FC0020E40704D5A9
:104060000721054A054806F093FD10BD4E63FF1F6A
:10407000FFFF0000593F001108BE0011A442FF1FBE
:1040800000B50C4BBFB01A780B4901A800F008FC32
:104090006B4680B25880002809D06A46074B6946B3
:1040A0001B881380064B0022188803F0D9FE3FB00E
:1040B00000BDC0462C63FF1F2D63FF1FFE42FF1F84
:1040C000FE43FF1F00B50C4BBFB01A780B4901A887
:1040D00001F00CFE6B4680B25880002809D06A4679
:1040E000074B69465B8D1380064B0022188803F04E
:1040F000B7FE3FB000BDC0465663FF1F5763FF1FAA
:10410000A442FF1FFE43FF1FF7B50E00377A1C00C5
:1041100008AB11003D001A8820231D401F423CD1EE
:104120003378022B3BD173681F785B781B023B43CB
:104130001E4FBB4208D01E4FBB4214D01D4DAB4298
:1041400021D00A252800FEBD002A2AD1142C2AD805
:104150002200F06807F0E0FC174B1C70012CF1D92D
:10416000FFF7B0FFEEE7002A1BD1202C1BD822005E
:10417000F06807F0D1FC114B04211C70104B18782B
:1041800007F0C2FCDEE7E3B20124009201940A00CA
:10419000310007F019FA0500D4E70825D2E7012518
:1041A000D0E70B25CEE70D25CCE7C046F3FF000096
:1041B000F4FF0000022900005663FF1F2C63FF1F5D
:1041C000D863FF1F10B5024804F0CCFC10BDC046F8
:1041D000893F001170B5160004AA148805AA157845
:1041E0004A685078117800022A4A08438018052846
:1041F0004BD807F0C1FC03131E29343F0720032CC2
:104200000BD80422121BAA4200D92A0022491A8084
:104210003000091907F080FC002070BD0720112C28
:10422000FBD81222121BAA4200D92A001B491A806D
:10423000EEE707200E2CF0D80F22121BAA4200D95D
:104240002A0017491A80E3E70720032CE5D8042247
:10425000121BAA4200D92A0012491A80D8E7072067
:10426000032CDAD80422121BAA4200D92A000E49D4
:104270001A80CDE70720032CCFD80422121BAA42B4
:1042800000D92A0009491A80C2E700220A201A80B0
:10429000C3E7C046DCD5FFFF53BE00117463FF1FA8
:1042A00043BE00113EBE001139BE001134BE0011E4
:1042B00010B50D21024A034806F06AFC10BDC04645
:1042C00028BE00111443FF1F37B5002000F0CCF8C2
:1042D000204D214BEA89287C9A422AD1042201A947
:1042E00000F076F9040000F033F9002C30D16B4671
:1042F00099882B68C9BA4B432989184A1B145B1843
:1043000053806B46D9886B6849BA89B24B43698937
:104310001B0C5B181248191C1BB2834200DD011CE8
:104320000B0400D5002113889180013313802000F5
:104330003EBD0223002101AA00F01CF96A460400D8
:1043400002230121287C063200F014F90443CAE755
:104350000124ECE78863FF1F83050000A063FF1FB3
:104360000F27000037B5012000F07EF81F4D07220F
:104370006946287C00F02CF9041E33D16B461B786B
:104380007F2B2FD800F0E4F86B46D878F023020496
:104390001B031A406B469B8815495BBA9BB21A43B4
:1043A0002B68000953432A891B0C9B184B806B46D2
:1043B0005A789B7812031B011A436B6802435343DC
:1043C0006A891B0C9B180B481A1C1BB2834200DD28
:1043D000021C130400D500220B888A8001330B8055
:1043E00020003EBD00F0B4F80124F9E78863FF1F08
:1043F000A063FF1F0F27000010B50F4C237C002B7C
:104400000CD0382B0BD1012000F02EF8CC22AC219F
:10441000207C920100F028F900F09AF810BD074BBB
:10442000E2899A42FAD1012000F01EF80021207C96
:1044300000F0FAF8F0E7C0468863FF1F830500002C
:1044400010B5084B1A7C002A09D05B69002B06D0F6
:104450009847041E01D0FEF7D3FD200010BD0124B3
:10446000F9E7C0468863FF1F70B5002106001620DB
:1044700006F078F80121152006F074F807F06CFBBF
:104480000400092007F028FA00222B4B2B4DDA6696
:1044900061321A6019685B3A9143002E28D0023AC3
:1044A0000A431A60AC4209D10A22DA6107321A6261
:1044B00000221A639A630132DA6370BD204A944283
:1044C00003D11E22DA610532F1E71E4A944203D17C
:1044D0003022DA610632EAE71B4A944203D14322D2
:1044E000DA610832E3E7194A9442E1D16922F7E739
:1044F00002220A431A604622AC4203D0104A944278
:1045000004D194225A6106329A61D1E70D4A94424D
:1045100001D1E622F6E70C4A944204D13422FF325C
:104520005A610D32F0E7094A9442C1D1E6225200A5
:104530005A610A32E8E7C046005000400024F40007
:104540000048E801006CDC020090D00300D8B805F8
:1045500010B50024064B0920DC6607F07DF9210028
:10456000162005F09BFF2100152005F097FF10BDD8
:1045700000500040F8B51C000023134D0F00EB66FF
:104580006860160007F070F901238022EB662300B3
:104590002F615200013B08D207F08EFB08200B4A26
:1045A0001168002C03D12000F8BD2A61F2E72B6FBF
:1045B000034203D02B69013C3370013613685B1A48
:1045C000032BEED90124EEE7005000406008FF1FE6
:1045D000002370B5124D1400EB6668600E0007F002
:1045E00043F901238022EB6623005200013B08D2ED
:1045F00007F062FB08200B4A1168002C03D1200051
:1046000070BD2A61F2E72B6F034203D02B69013C96
:104610003370013613685B1A032BEED90124EEE7E1
:10462000005000406008FF1F002370B50C4C0D00C7
:10463000E366606007F018F90123E366256107F07F
:104640003BFB8020074A80001168636B034205D161
:1046500013685B1A032BF8D9012070BD0020FCE71A
:10466000005000406008FF1F002370B5134C0E007F
:10467000E3666060150007F0F7F80123E366266142
:104680000F33626B1A42FCD02B0A23611023626B3A
:104690001A42FCD0EDB2256107F00EFB8020084ADB
:1046A00080001168636B034205D113685B1A032B0A
:1046B000F8D9012070BD0020FCE7C0460050004042
:1046C0006008FF1F002370B5124D0C00EB66686098
:1046D000160007F0C9F80123A619EB660F33B442A0
:1046E0000ED107F0E9FA80200B4A800011686B6B4D
:1046F00003420CD113685B1A032BF8D9012070BD5B
:1047000022782A616A6B1A42FCD00134E7E7002064
:10471000F5E7C046005000406008FF1F10B5084C88
:10472000E368002B08D1074B1B685B045B0C0A3362
:104730006360054B1B68236007F006F8A06010BD9E
:10474000C863FF1FC8F00040CCF0004010B507F070
:104750008BF80F4B996A9A6A8A42FBD10D4C6268BA
:10476000A0688A18121A531E884200D31300A16051
:104770002168DA0B52185B0407495B0C6360226006
:104780000B60064B1A6007F097FA206810BDC04610
:1047900000F00040C863FF1FC8F00040CCF00040AC
:1047A00070B51D4C23793F2B01D93F2323711B4B3F
:1047B00022791A701878C0B207F0B6F81823184991
:1047C000184A0B80184913800B805380A37917492E
:1047D00080200B800C21938001334B430001191C76
:1047E000834200D9011C124BD18019806379002BC0
:1047F00001D101336371237A012B01D80223237283
:104800006279237A0B4853430A21584307F04CF945
:10481000094D286070BDC046BC63FF1F480AFF1FDA
:10482000FC43FF1FC845FF1FFA43FF1FA865FF1F7A
:10483000F843FF1F71020000AC63FF1FF8B51121A0
:104840000020FEF7C3FD114C011E114D09D10C22B1
:10485000104BC1CBC1C4280007F0FEF9FFF7A0FF41
:10486000F8BD0C2220000C49FEF784FD0C2802D074
:10487000084B43CB43C40C2228000849FEF77AFDBD
:104880000C28EBD00C220021E5E7C046BC63FF1FDB
:104890008863FF1F94BE0011FC0C0000F50C0000A3
:1048A000F0B5002604000D0085B0B2426AD04B1C62
:1048B000087801934B7889782F7909021943EB78AE
:1048C0003F061B040B431F43039720706670262886
:1048D00000D192E01CD8102812D806F0F5FF4D0048
:1048E000FF003300330033009700A5009E00330023
:1048F0003300330033003300330033003300E5006E
:10490000232800D1BFE025285FD0FF2363709AE001
:10491000602800D1A2E00CD8552836D056284ED0B9
:104920003328F2D10A229B49601C07F0F5F80B26C8
:1049300028E0722800D188E0DC2800D1EDE0712861
:1049400000D178E0DB2800D002E1042ADDD910266E
:10495000052A05D0561F32003800691D07F0DCF823
:1049600005222900200007F0D7F832003900601D29
:1049700007F0D2F8053605E00C222000864907F042
:10498000CBF80C26300005B0F0BD013A834D0C2A5F
:1049900013D8002A0AD02800019907F0BDF8FFF7C4
:1049A000FFFE0C2228007E49FEF71EFC0C22290087
:1049B000601C07F0B1F80D26E4E70C22EBE7774D19
:1049C000784B2A0043CB43C2E9E7013A764D0C2AE3
:1049D00011D8002A08D00199280007F09DF80C2270
:1049E00028007249FEF700FC13222900601C07F022
:1049F00093F81426C6E70C22EDE76B4D1322310025
:104A0000280007F029F9FEF7FBFAEDE705226849CF
:104A1000601C07F081F80626B4E712226549601C85
:104A200007F07AF81326ADE708226349601C07F007
:104A300073F80926A6E76978F72900D965E75F4B7F
:104A4000188801F0AFFD02269CE75D4B012A03D0D8
:104A50006A785A706270F6E75B7857E7013A594D09
:104A6000062A0ED8002A05D00199280007F054F82C
:104A700001F016F806222900601C07F04DF8072601
:104A800080E70622F0E7042A04D94F4D2F6006F094
:104A90005BFEA860FFF75AFE0422039003A9601C86
:104AA00007F03AF805266DE7484D062AE2D90622B6
:104AB0002800019907F0F8F80028DBD006220199B8
:104AC000280007F029F8062241492800FEF78CFB50
:104AD00001233B4A51780B435370CBE7931E3D4F64
:104AE0001A2B04D86B78002B09D100F021F93A4B2E
:104AF00039001E78601C721E07F00EF842E7551E42
:104B00002A000199380007F007F83449AAB23800A2
:104B1000FEF76AFB00F042F9E9E7022A00D8F4E662
:104B20006B78BFB26370AB78A370032A05D0033AE9
:104B3000390092B2E81CFEF757FB10223900E01C46
:104B4000FEF718FCC61C002800DB1BE760707AE744
:104B5000DA2800D0D9E6042A00D8D6E6082A15D9E2
:104B6000AB796A791B021343EA7912041A432B7A50
:104B70001B0613433B603B6805222900200003937A
:104B800006F0CAFF0422601D03A950E7FE236370EC
:104B9000F1E7C046A063FF1FA0BE0011BC63FF1F6A
:104BA000FC0C000094BE00118863FF1FF50C000090
:104BB0009463FF1F7463FF1F3C45FF1FFE43FF1FED
:104BC000B863FF1F9944FF1FC863FF1F6509FF1FDC
:104BD000ADAC0000BB65FF1FB965FF1FAEDE000076
:104BE00070477047020010B5094B0A32094C92B267
:104BF000DA815A8298811882207802F039FB0422E7
:104C0000054B012120781A7006F07EFF10BDC046CA
:104C1000C644FF1F0666FF1F0566FF1F013870B5FB
:104C2000042809D806F0A8FF030925081200214B23
:104C30000221187806F068FF70BD1E4B0821187815
:104C400006F002FF00221C4B1A72F5E700241A4BF3
:104C5000184D1A68082128781C8107F045F82100B2
:104C6000287806F079FD012000F052FE00F018FFD0
:104C7000E2E7104B0821187806F0E6FE0F48FFF730
:104C800007F90F4B0F4A9B79002093800E4A13803F
:104C90008022094B52001A8100F03AFE00F000FF1A
:104CA0000A4B5B78002BC7D0094A136006F0BCFEA4
:104CB000C2E7C046D863FF1FAC63FF1F0744FF1F56
:104CC000BC63FF1FC845FF1FA865FF1FB863FF1F18
:104CD00034F0004010B5012909D1054B1B78002B99
:104CE00005D02622034B04485A72FFF77BFF10BD04
:104CF000DC65FF1FAC63FF1FC40900000300F0B5B3
:104D00000A4D8E18B14202D152008018F0BD0C78C5
:104D10002F6824093C5D0F271C700C7801313C4042
:104D20002F683C5D5C700233ECE7C046F443FF1F24
:104D30000D22114B10B51A700C23104C1049237022
:104D4000093A033B0F48637006F0E6FE2D2301226B
:104D50000D490E48A371FFF7D1FF01220C49FFF75F
:104D6000CDFF01220B49FFF7C9FF00220A491000BD
:104D7000FEF73AFA10BDC046D865FF1FB965FF1FA0
:104D800053BE0011BB65FF1F6709FF1FC065FF1FF2
:104D90006609FF1F6509FF1FAEDE000070B5124CEB
:104DA000132220001149FEF7E5FA114D002817DD06
:104DB000AB78002B14D0431C2B7009236B7000239D
:104DC00000190370287829000130C0B206F034FFC2
:104DD000297822000139C9B2002005F0F7FD70BD25
:104DE000FFF7A6FFEEE7C046BB65FF1FAEDE000083
:104DF000B965FF1F10B5114B1A781870002A0ED034
:104E000000280BD10E4B1A78062A07D85423D3401A
:104E1000DB0703D50B4B187802F02AFA10BD0028E7
:104E2000FCD0074B1B78012B02D0033B022BF5D89B
:104E3000044B0121187806F067FEEFE7DC65FF1FE1
:104E40000566FF1F0666FF1F70B5504E504A514958
:104E50003070082005F046FC0121022005F04CFBD3
:104E6000022005F02DFC0121002005F045FB00206B
:104E700005F026FC00F0DEFEFEF7C2F806F084FE28
:104E8000032245494548FFF739FF2D24030004223A
:104E90001C7043490130FFF731FF30230470414D4E
:104EA000414C437083702E3B062220003F49EB8724
:104EB000FEF760FA062813D0200006F0FDFD022858
:104EC00009D00321200006F0DFFE8D23E3706E3B46
:104ED000237119336371062220003449FEF784F9E7
:104EE000334B1B68FC335C64FFF758FF0020FFF76F
:104EF00081FF304C304A0121304B1278207802F08B
:104F000079F92F4A2F4B12780021207802F072F99C
:104F100001222D4B1A702D4B9B78552B31D12C4BE8
:104F20003B325A722B4A2C4BAA81EB812A826B822C
:104F30002021307806F008FD0120404205F092FD66
:104F40000120404205F02EFEFFF7B2F9FEF784FF84
:104F500000F092FC01204042FFF776F8012006F0B5
:104F6000D3FCF72001F002FB0121307806F0CCFDE4
:104F7000307802F0D9FA194806F0F6FDFEF77AFE0D
:104F800070BDFA22164B5201CEE7C046D863FF1F10
:104F9000E14B0011D54C00113C45FF1F7463FF1F0E
:104FA0009463FF1FC644FF1F6509FF1FADAC0000DF
:104FB0006466FF1F0666FF1F2644FF1F0744FF1F8E
:104FC000D865FF1FB965FF1FAA65FF1FB863FF1FE4
:104FD000AC63FF1FC4090000CE090000DA63FF1FA5
:104FE0004A1F0000F8B50A0020230D001A4019429C
:104FF00047D04F4B1B78002B40D0FFF7A7FB4D4B02
:105000004D4C4E4E99686268737A8A1ADB039A4255
:1050100002D36160FEF72EFE327A217A531EDBB294
:10502000994205D1FFF7E8F9002000F0EBFD0FE011
:105030009142F9D300232372FFF702FA012000F016
:10504000E1FD3F4F3800FEF723FF390006F084FCF6
:10505000637A002B0FD0013BDBB26372002B0AD1C5
:10506000384B9B78552B01D106F0DEFC6423707918
:105070005843FFF7B7FD237A01332372202068409D
:10508000F8BD0BB2002B0ADA2F4B187806F0ACFDF6
:10509000002801D006F080FB80200002EFE7022408
:1050A000214206D0244B01201A72FFF7A3FE2000F4
:1050B000E5E70B071ED5FFF749FB1E4B1E491F4CAA
:1050C00098684A68637A821ADB039A4202D348607E
:1050D000FEF7D0FDFFF7B4F9FFF78EF9012000F0DD
:1050E00091FD00F0E3FB2368DB0701D5FFF76AF8C9
:1050F0000820C4E71024214206D00D4B1B78002B5A
:10510000D5D1FEF7BDFED2E70124214207D00F48DA
:1051100000F06AF806F0B0FB00F0EAFCC7E70424F0
:10512000080020402142ABD0FEF7AAFFBFE7C046EF
:10513000DC65FF1FC863FF1FAC63FF1FBC63FF1F5D
:105140000744FF1FB863FF1FD863FF1FEC43FF1F17
:10515000F0B51B4B1B4F1B883A8804001A4E1B4DA1
:1051600085B09A420DD832889A420AD3184B1A88D1
:105170002B889A4205D1174A174B12881B889A42EE
:105180001BD0052001F048FA3B8802AA138033881F
:10519000019053802B88114D93800F4B02A91B88DF
:1051A000D3800F4B2A78188802F064FF0D4B08213A
:1051B0002878019A1C7006F00FFB05B0F0BDC046C0
:1051C000A665FF1FFC43FF1FFA43FF1FA865FF1FD3
:1051D000A465FF1FA265FF1FF843FF1F0666FF1FA0
:1051E000FE43FF1FA065FF1F13B50C4B1C78002C5E
:1051F00011D1002801D00A4B18600A4A0A4B1178D5
:105200000A4A10780A4A01920A4A0092002205F0DE
:10521000D5FA200016BD1124FBE7C0460566FF1F26
:105220009C65FF1F0466FF1FF465FF1F0666FF1FD6
:10523000E065FF1FE465FF1F10B5064B12201B78C9
:10524000052B06D1044B13221988044B187801F062
:10525000BFFB10BD0566FF1FFE43FF1F0666FF1F55
:1052600010B500240122114B52421870104B1C70D3
:10527000104B1A8002F058F904220F4B21001A70CB
:105280000E480C3206F0E0FC102221000C4806F01B
:10529000DBFC07220B4B1C600B4B1C700B4B1C7078
:1052A0000B4B1A700B4B1C7010BDC0460666FF1FDF
:1052B0000566FF1FFE43FF1F0466FF1FF465FF1F07
:1052C000E465FF1FE065FF1FB865FF1FB765FF1F9F
:1052D0000044FF1FB665FF1FF8B5174C0600257880
:1052E00006A814240078052D23D1B41F134FA5B2AE
:1052F0001824BD421DD88D1FADB2BD4219D8FA2564
:105300006D00AA4215D21D000D4F0A3DADB2BD423F
:105310000FD80C4C26800C4C21800C4900240A80AC
:105320000B4A1380FFF714FF0A4B0421187806F08C
:105330008BFB2000F8BDC0460566FF1F790C0000FE
:10534000750C0000FC43FF1FFA43FF1FA865FF1FF9
:10535000F843FF1F0666FF1FF0B50BB20D0089B0C2
:10536000002B00DB70E1A44E307806F03DFC041EFB
:1053700050D00378A22B00D122E1D02B1AD0912B50
:1053800045D143780E2B42D19C4B82889A423ED124
:105390009B4A83681278052A39D1032018567F2842
:1053A00035D0984B1B68002B31D05B68002B2ED07A
:1053B00098472CE08078072829D806F0DDFB0428E0
:1053C000183F3F74A8D86378002B0CD101218C4B77
:1053D00019708D4B1A78002A5BD08C4B307801F015
:1053E00009FF002855D00722854B1A7051E06178DB
:1053F0000029F8D1E378002B11D0854A854B12782B
:10540000307801F0F7FE60706378002BEBD120005C
:1054100006F0C2F980200002684009B0F0BD784B68
:105420001B78022BF3D00121307806F0CDF900284B
:10543000EAD10121307806F067FBE5E76378002BBD
:10544000D1D16F4F032807D13B78052B02D101330F
:105450003B701EE00223FBE76F4B1A886F4B0293F1
:10546000002A0BD01B78002B03D00121307806F0E6
:10547000B3F93B78062B04D1013BE9E7029B1A7094
:10548000F7E7042B41D10121029B3078197006F017
:105490003BFB5C4B1B68002BB9D01B68002BB6D0C4
:1054A000574A107884E76378554F002B27D106229E
:1054B000211D5B4806F030FB62895A4B5A491A801D
:1054C000A2895A4B1A80E3890B800521397058490B
:1054D0000A80584A1380228A574B1A80574B1B78F0
:1054E000012B09D11F2001F097F8FA2292004243C4
:1054F0000421307806F070F90022484B75E7312B13
:1055000000D070E70022454B1A700323A0E7062263
:105510000021434806F098FB0023454A04211380EC
:10552000444A30781380444A138006F08DFA0821EB
:10553000307806F089FAA379083B5A425341304A41
:1055400003331370304B1B78002B06D0334B30786D
:105550001A78002A06D001F08BFE0122314B52420C
:105560001A8096E70121197006F0CEFAF5E70821B6
:10557000307806F069FA6378002B00D047E72C4BAF
:105580002D4F0293E388029A04211380294B30782F
:1055900003932389039A138063893B8006F014F9EF
:1055A000002800D033E7264B1B68002B00D12EE7E4
:1055B000039902983A88098800881B68984726E76B
:1055C0004379132B00D022E70389012B0AD11D4B0D
:1055D0001B78022B06D10821307806F035FAFFF748
:1055E0002BFE14E7052001F017F80821020030789F
:1055F00006F0F2F80BE7C0460666FF1F0514000030
:105600000566FF1F9C65FF1F2644FF1F0744FF1F01
:10561000D865FF1FB965FF1FDA65FF1FDC65FF1F37
:10562000AB65FF1FFE43FF1FB265FF1FB465FF1F81
:10563000A665FF1FA465FF1FA265FF1FAA65FF1FC8
:105640009865FF1FA065FF1F8020C001014200D0A8
:10565000E2E6CB0731D5324B1B78002B1DD0314E03
:1056600005AC3378052B1AD1023B23702E4B210059
:105670001B7823722D4B1B7863722D4B187801F029
:105680005DFD002809D007202A4B30701B68002BD5
:1056900003D01B68002B00D098470120BCE60E20E9
:1056A000254B06221B7825492370254B1B786370F8
:1056B00002ABC01806F030FAD8E702230800184001
:1056C000194209D0174B1B78052B03D11D4B1888A5
:1056D00006F0CAF902209FE60424214203D0FFF716
:1056E00037FD200098E6082308001840194200D131
:1056F00093E6154B1C78012C03D0022C0DD008200A
:105700008AE6124B124A134913481B8812880988EB
:1057100000880094FFF7E0FDF1E7FFF78DFDEEE76D
:10572000DC65FF1F0566FF1F0044FF1FB665FF1FF6
:105730000666FF1F9C65FF1FB865FF1F0144FF1F22
:10574000B765FF1FFE43FF1FA065FF1FF843FF1F44
:10575000A865FF1FFA43FF1FFC43FF1F10B502A8F7
:1057600004880B20002C10D1496808784978090278
:1057700001430C48814209D1022119800A4B598802
:105780001170DB7800205BB2537010BD074C0A200B
:10579000A142FAD102211980034B998811705B79DB
:1057A000F0E7C0466E2A0000A063FF1F6F2A0000CA
:1057B000F7B5150008AA16884A680F4F1478527872
:1057C000120222430A24BA4214D10122DBB201920E
:1057D00000962A0005F0F8FE041E0BD1074B1B684B
:1057E000002B07D068782A780002104342425041CB
:1057F000013098472000FEBD022900001866FF1FF7
:1058000030B5012503790400BFB02B4227D01549DC
:10581000408805F045FA28420DD06A46124B694689
:105820005B8D138002235380104B5B8893806088CC
:10583000002202F015FB0E49608805F031FAC0071E
:105840000DD56A460B4B69461B8813800223538093
:10585000064B9B8893806088002202F001FB3FB0DA
:1058600030BDC0461066FF1F2844FF1FA063FF1F06
:105870000866FF1F8244FF1F10B5074C0749200030
:1058800005F0C4F92000064905F0C0F90721054AD2
:10589000054805F07DF910BDFFFF00001066FF1FF1
:1058A0000866FF1F20BF00112844FF1F10B50248E3
:1058B00003F058F910BDC0460158001170B55F25BE
:1058C000082607498400CA788B7840012A40B343F0
:1058D0003440A843234302438B70CA7070BDC04656
:1058E0009944FF1F010043B204205A0002409B006C
:1058F0000C3003401A43152310B5044CE07898434C
:10590000143B0B4018430243E27010BD9944FF1F43
:1059100010B5054B082419790A00A243002801D0CC
:1059200022000A431A7110BD9944FF1F10B5054BA0
:105930004024D9780A00A243002801D022000A435B
:10594000DA7010BD9944FF1F0821F8B5324D334B72
:10595000AE7804000E40AE70984204DD67232B70D1
:10596000473B6B70F8BD2E4B984203DAE0232B7057
:105970003A3BF6E700232B706B7083B21A0029487C
:105980005F3292B2284F82422CD9002C03DA5B425C
:105990001CB204232B70053420B20A2106F084F8CF
:1059A00004B2FA239B009C4232DB08232A7813437B
:1059B0002B706421200006F077F80A2100B206F06F
:1059C00083F809B22A787B5C13432B700A212000EC
:1059D00006F06AF80A2100B206F076F809B27B5C9C
:1059E0006A780AE06970002CDBDA5B421CB204239F
:1059F0002B70F3226B78092CE8DC13436B700A21BF
:105A0000200006F061F809B27B5C1E43AE70A9E786
:105A1000632CCEDCEDE7C0469944FF1F1B4E00000F
:105A20001DFCFFFF2A0800004ABF00110823F7B53C
:105A3000194FCD003E7904001E403E71EDB263283F
:105A400006DD5F3333433B7120231D437D71F7BD7A
:105A50000300093305DA20235B4233433B71A6235D
:105A6000F3E70E4B019300280BDA0423444224B2DF
:105A70003B710A21200006F027F8019B09B25B5C0C
:105A8000E3E70928F5DD0A2106F00EF8019B00B2D4
:105A90001B5C1E433E71ECE79944FF1F4ABF001197
:105AA00070B50F4B1B78002B18D00E4E0E4D0622F2
:105AB0003100280006F0F8F800280FD00622310047
:105AC0000A4C280006F028F80120FEF7CDFC07223A
:105AD00021003E20FEF7F6FDFEF73AFD70BDC04600
:105AE0002366FF1F9944FF1F1D66FF1F1C66FF1FD3
:105AF000E622402110B5094B1A70403A5A703E32E6
:105B00009A70DA780A40DA701A7938390A40053919
:105B10000A431A715971FFF7C3FF10BD9944FF1F63
:105B2000F8B51C4B3C21186805F04EFF3C210400E1
:105B300005F0E2FD20000F003C2105F045FF182193
:105B400005F0DAFD00230E00134C0A21237030000B
:105B500005F03AFF114D0A212B5C3000637005F00F
:105B6000CBFD40226B5C2679A370E37838001340AC
:105B7000E37008230A211E4005F026FF2B5C0A2152
:105B80001E433800267105F0B7FD6B5C6371FFF7AB
:105B900087FFF8BDC863FF1F9944FF1F4ABF00116C
:105BA00010B5164C0A210223E05E05F07DFF00B21D
:105BB000FFF7CAFE0423E05E642105F075FF0121B2
:105BC00000B2FFF733FF237A0024132220009A4209
:105BD0006041C0B2FFF7AAFE0320FFF76FFE20006E
:105BE000FFF780FE064B1878053843425841C0B293
:105BF000FFF78EFEFFF754FF10BDC046A063FF1FE6
:105C00000566FF1F094B10B51B689B0708D5084A9E
:105C10001378591C1170DB0704D5FFF781FF10BD05
:105C20000028FCD0FFF7BCFFF9E7C046BC63FF1FAC
:105C3000B863FF1F002010B5FEF716FC10223E20AF
:105C40000549FEF73FFD0023984200D13E33034A49
:105C50001370FEF77DFC10BD3ABF00112366FF1FD5
:105C60000200F0B501270A480A4E51188B1A002B82
:105C700000DCF0BD08241578430868403840400037
:105C8000805B013C58406D08002CF5D10132EDE7F6
:105C9000FFFF00005ABF0011F0B500250F269D42FE
:105CA00000DBF0BD4C5D070944403440A400A0581F
:105CB00001357840F3E70000F0B589B06A460D0081
:105CC0000B000F27110010351C7801332600240922
:105CD0003E40167054700232AB42F5D12023024A86
:105CE000FFF7DAFF09B0F0BD60BF0011F0B54E78E4
:105CF0000B7889B036020C00170001901E43012A70
:105D000061D9954B9E4200D877E001339E421CD169
:105D1000062A17D1CA788B7812021A430B791B0412
:105D200013434A7912061A438C4B5A6100221A70A7
:105D30005A808B4A5A608B4A9A608B4ADA600020FC
:105D400009B0F0BD88225205EEE7884B9E423CD157
:105D500082498B78002B00D0F6E00C2A31D10F223B
:105D6000A3789343E2781202134322791204134377
:105D70006279120613434B60E279A0791202024362
:105D8000207A00041043627A12060243CA60E27A63
:105D9000A07A1202024376484A81834208D804233B
:105DA0006E49142201980B7005F0B6FE1420C7E767
:105DB0001201D21889235B059A42F0D801238B7017
:105DC000BDE7022AFAD00523EAE76A4A0123964290
:105DD000E6D1FFF731FA052F0CD9E378A2781B0240
:105DE0001343227912041A4363791B061343624A50
:105DF0000393136005F018FEA1E7584D2B78002B94
:105E00009DD1AB78002B00D1A0E02B8901339BB250
:105E10000093B34200D091E0132AD4D9CF7C8B7C7D
:105E20003F02122120001F43FFF71AFF874200D0D4
:105E30008EE0002E3DD1E378A2781B021343227935
:105E4000E96812041A4363791B06134303930A2279
:105E50008B4212D1FF23A370E370237163716B89AE
:105E6000002B09D1E37B227C1B0212041343A27B8B
:105E700013431B0901336B8100226B89002B8ED0E9
:105E8000002A67D1686837013818000B6B69000376
:105E90000390984205D9686105F006FDEB7801335F
:105EA000EB7068681022A11C381805F025FD2E81C2
:105EB00045E76F89009A7B1E9BB293423AD1E27804
:105EC000A37812021A43237905A81B0413436279AD
:105ED0006C6812061A43EB6800920392211D0C2293
:105EE000049305F019FE0120260004A94042103653
:105EF000FFF7E2FE013F012F17D1009A0B23286123
:105F0000824200D04CE704221C49200005F0F4FC3A
:105F1000042203A9686805F037FCE968039AFF23A7
:105F2000914200D13CE7F73B3AE73100FFF7C4FE6E
:105F30001036DFE70923B742A4D831E7009BB3420C
:105F400000D9FCE607232BE7022329E7032327E7F1
:105F5000062325E70A2323E7FFFE0000A044FF1FD6
:105F600000000111FFFF00005048593601FF0000FA
:105F7000FFFF001102FF000034F00040AC44FF1F9F
:105F800010B5034C0B000122210000F06BFA10BD8C
:105F9000416100110B8870B506000D000224162B1C
:105FA00011D92B000322094900F05CFA041E0AD122
:105FB000074B2A881B88191C934200D9111C3000FA
:105FC00089B200F0EFFA200070BDC0466D6100118B
:105FD0007E66FF1F10B54A780400013A0B000220CC
:105FE000012A07D80A78002A04D005222000024995
:105FF00000F038FA10BDC0469B6100110A7810B558
:106000000B0004000220002A04D0072220000249CD
:1060100000F028FA10BDC046476200110A7810B59A
:106020000B0004000220002A04D0092220000249AB
:1060300000F018FA10BDC046AD62001110B5034C57
:106040000B000B22210000F00DFA10BDDD620011E3
:1060500010B5034C0B000D22210000F003FA10BD17
:106060004F63001110B5034C0B000F22210000F00C
:10607000F9F910BDA96300110A7810B50B000400EE
:106080000220002A04D011222000024900F0EAF97F
:1060900010BDC046B9630011002310B513221900CA
:1060A00000F0E0F910BD000010B5034C0B00172202
:1060B000210000F0D7F910BD0B640011002310B5CA
:1060C0001922190000F0CEF910BD000010B5034CE4
:1060D0000B001B22210000F0C5F910BD4564001122
:1060E000F7B584890D0006000121002C22D0002381
:1060F0008268D3561778002B1EDA0C2C1AD90C3C68
:10610000A4B2131940880093230002F086FE431EB8
:10611000984101307B06DB0F6B703F23013C1F4031
:10612000A4B22870AF70AC80002C07D0B3680133E4
:10613000AB6000210800FEBD0020EBE7AC60F8E793
:106140000B7803704B8843704B881B0A83700B7964
:10615000C370042070470420022B06D1002053781E
:1061600011781B02009A0B43138070470B88037051
:106170000B881B0A43700220704704200099834259
:106180000AD1537810781B0203430B80D3789078A0
:106190001B02034300204B807047F8B50D004B787D
:1061A00001240021461C03702B788B4201D820006B
:1061B000F8BD6B78B01C4F1C012B10D189006918F9
:1061C0004B88022233704B88B9001B0A7370691820
:1061D00005F052FD04360434A4B2F9B2E4E7122308
:1061E00059436B185A88043132705B8810221B0A9D
:1061F0007370691805F040FD12361234ECE770B583
:10620000049D14001E00052B01D8042070BD637886
:1062100012781B0213432B80E378A2781B021343EE
:1062200002226B802A71211D681D063E05F024FDA7
:10623000B2B22A81F02AE8D82800A11D0A3005F060
:106240001BFD0020E2E7002310B50A789A4201D82E
:10625000900010BD9A008A18548801330470548845
:10626000DBB2240A4470948884709288120AC27047
:106270000430EAE710B51100029C062B04D004207C
:106280001022142B01D010BD022222714B78087805
:106290001B0203432380CB7888781B02034363806F
:1062A0000431601D05F0E8FC0020ECE710B50C7827
:1062B0008B7804315C43E4B203702200013005F0B6
:1062C000DBFC601C10BD0420022B06D1002053789B
:1062D00011781B02009A0B431380704710B50C0015
:1062E0000A88023105F0C8FC208810BD70B5040092
:1062F0000D0004981100012B01D8042070BD167800
:1063000052781202324302800200F8325570147043
:10631000E825002C00D10C35023B9AB24280AA42FB
:10632000EBD80231043005F0A7FC0020E6E704209A
:10633000009983420AD1537810781B0203430B80E3
:10634000D37890781B02034300204B80704710B530
:106350000C000A88023105F08FFC208810BD000077
:1063600070B501211E000420049C0E400B4218D180
:10637000CB40DDB28D4214D90A49DBB2098899427B
:106380000FD32300F6331D703300580011184978DD
:10639000165C0902314301332152D9B28D42F4D83F
:1063A000002070BDC044FF1F10B50C000A880231E8
:1063B00005F062FC208810BD10B50C788B78043194
:1063C0005C43E4B203702200013005F055FC601C10
:1063D00010BD10B511000298032B01D8042010BD88
:1063E00014785278043B120222430280CA788C78D7
:1063F0001202224342809AB28280F22AEED80431FD
:10640000063005F039FC0020E9E710B50C000B88D8
:1064100003700B881B0A43704B8883704B881B0AE0
:10642000C3708A880430063105F026FCA088043049
:1064300080B210BD0420012B03D100201378009AF4
:106440001370704710B50C000B8803700B881B0A83
:1064500043704A880230043105F00EFC6088023037
:1064600080B210BDF0B589B003931E4B029242007A
:106470000700D05A019102F020F81325061E2DD0F6
:10648000029B01240370019B002B04D00019039987
:106490009847001984B26B461B7A5BB2002B0FDA67
:1064A0001021380002F01CFB1925002813D1300000
:1064B0003219E1B202F066FC051E0CD10C34A4B214
:1064C000042304AA380005A993800696948101F05C
:1064D000AFFD051E02D0300005F04EF9280009B0CE
:1064E000F0BDC0467C66FF1F70B505000C0000289B
:1064F0000CD00020814209D010222000044905F070
:10650000BBFB01202B7823736B78637370BDC0468F
:10651000A0BF0011F0B506000D0017001C0085B0EB
:1065200002291BD00020102907D1022B07D0102BE5
:1065300003D115E00020102C08D005B0F0BD69464D
:106540003800FFF7D1FF2A0069460BE069463000AA
:10655000FFF7CAFF22006946380004E0022BE9D1A8
:106560002A003900300005F01FFBE6E7031CF7287E
:1065700000D9F723032008499AB2013A0B80D317B8
:10658000034006499B189B100B80D30F04499B18AE
:106590005B100B807047C046C444FF1FC244FF1FFE
:1065A000C044FF1F034B1B888B4202D3024B4000A9
:1065B000C1527047C444FF1F7C66FF1F014B40005F
:1065C000185A70477C66FF1F1722014B1A807047CC
:1065D0007C66FF1F70B505000E2005F0EDF9041E66
:1065E00013D0D0230370002306228370074945701F
:1065F000033005F041FB064B2100DA8A62811B7EE5
:106600002373044B187805F0CFF870BD9866FF1F10
:106610008866FF1F1445FF1F262803D8024B400041
:10662000C05A70470148FCE7C644FF1FFFFF000047
:1066300070B506000C00094D1C220021280005F051
:1066400003FB074B1E70074B1C7005F09DF90123DF
:10665000002801D0002312202B7070BD8866FF1F18
:106660001445FF1FA966FF1F70B505000D4C0800FB
:10667000E260A16010220021656005F045FB012861
:1066800003D11021A06802F058FD1022002128003B
:1066900005F03AFB012803D11021606802F04DFD9E
:1066A00070BDC0468866FF1F70B5041E05D1002965
:1066B00003D006220D4805F0DFFA0D4B1D78012DA1
:1066C00011D1002C05D102221A7005F055FB2800CB
:1066D00070BD00221A70074B1B78FF2BF7D02000EB
:1066E000FFF778FFF3E70025F1E7C0469866FF1F44
:1066F0008866FF1F1445FF1F030010B5002801D155
:10670000002010BD00780B4A002803D15988D1829F
:106710001B7913761378022BF2D10023984200D113
:1067200003331370044B1B78FF2B01D0FFF752FF8C
:106730000120E6E78866FF1F1445FF1F002911D0DE
:1067400000280CD04B79012803D140225242134338
:1067500003E03F221340032802D001204B71704711
:106760004022F4E70800FAE770B5094D01002878E7
:1067700000280BD0074C0622200005F07DFA2100EE
:106780002878FFF7DBFF200004F0BEFF70BDC04695
:10679000A866FF1F8266FF1F00290AD0012808D1C2
:1067A0003F224B799343C02B03D0403B5A42534185
:1067B000981C704770B5174D06002B78FF2B15D02D
:1067C0000A2005F0F9F8041E10D0D0230370C83B4E
:1067D0008370114B11491B784670C3700622043038
:1067E00005F04AFA2100287804F0DEFF0C4B1B78F4
:1067F000012B0DD10B4B1B68002B03D09B68002B8A
:1068000000D09847084B04211878084A05F06CFA24
:1068100070BDC0461445FF1FA866FF1F8266FF1F9C
:10682000A466FF1FD066FF1FD466FF1F60EA00004A
:10683000014B98687047C0468866FF1F014BDB68B4
:10684000186870478866FF1F074B10B5DA68136831
:1068500001331360054B1878FF2803D08021C9014C
:1068600005F052F910BDC0468866FF1F1445FF1F92
:10687000F7B50E0002F0C8F8051E1CD00E4B0662DC
:106880001F78002F00D10778AB791020019305F015
:1068900093F8041E0FD0D0230380C73B8370019B65
:1068A000E91DC3700622043005F0E6F92100380026
:1068B000E66004F079FFF7BD1245FF1F014B187821
:1068C0007047C046A866FF1F054B002805D1054B41
:1068D0001A78054B002A00D1014B18007047C046BA
:1068E0009866FF1FA866FF1F8266FF1F014B58684E
:1068F0007047C0468866FF1F024B1868431E9841C8
:10690000C0B27047AC66FF1F421E03000120152A6B
:1069100003D9FF3B5A425341D8B27047F0B51C002F
:1069200000230E0085B0039002920B70029A9342EE
:1069300001D3002019E0E55C5A1CD2B2002DF8D03A
:10694000029851198142F4DC0233DFB2A35C1800D3
:106950000193FFF7D9FF002807D0013D019A039961
:10696000EBB233708A4202D1E01905B0F0BDDB19F9
:10697000DBB2DBE710B50C0002F09EF8030012203A
:10698000002B03D02100588805F0C6F910BD000087
:1069900070B50E4D84006359002B15D0186A00287D
:1069A00001D004F021FF2B59586A002801D004F0CF
:1069B0001BFF2B59986A002801D004F015FF2859B5
:1069C00004F012FF00232B5170BDC046B866FF1FB4
:1069D0001C4B70B504000E00150099420AD11A4BE9
:1069E0001B68002B01D1122070BD1B68002BFAD050
:1069F0009847F9E7154B994215D1134B1B68002BAB
:106A00000AD01B68002B07D09847002804D1104BF0
:106A10001C70104B1D70E7E729002000FFF7AAFF4C
:106A20000028E1D1F3E7080001F0EEFF0028DAD0FA
:106A300003780320A342D7D12900300005F06CF978
:106A4000D2E7C046FEFF0000B466FF1FFFFF000054
:106A5000B166FF1FB066FF1FF7B50400808801F024
:106A6000D3FF0025A84203D00578A08802F008F8DB
:106A70001C4E3378002B1FD0AB421DD11A4B28007F
:106A80001978FFF777FF002818D000233370A37917
:106A90000820A778A688019304F08EFF011E0DD070
:106AA000D0230370CA3B8370019B4770868083713B
:106AB000280004F079FE01E0002DE8D1A0880B4BFE
:106AC0008200D358002B01D0FFF762FF1721A08866
:106AD000FFF768FDA08801F027FDA08801F0FEFD0A
:106AE000F7BDC046B166FF1FB066FF1FB866FF1F47
:106AF000F0B587B01D000CAB1B88070001930DABF0
:106B00001B88142002930EAB1B88160003930FAB57
:106B10001B880091049310AB1B88059304F04CFF75
:106B2000041E1AD0D0230370CB3B47708370C6700D
:106B3000062229000430002D11D005F09DF8019B9C
:106B400021006381029B0098A381039BE381049B46
:106B50002382059BA37404F027FE07B0F0BD05F067
:106B600073F8ECE7F7B5009308AB1B8807000C201F
:106B70000D001600019304F01FFF041E13D028001F
:106B800001F042FF00280FD00078D0232370C93BCA
:106B9000A370009B21002381019B6770A580E68084
:106BA000638104F001FEF7BD014B1878EDE7C046A4
:106BB0001445FF1F13B5040064890389C2888188C6
:106BC000C0780094FFF7CEFF13BD000010B5044C51
:106BD0002068002803D004F007FE0023236010BDC6
:106BE000BC66FF1FA122F0B5818892004A43384B52
:106BF000384F1B6804009B189D2292009B188279D5
:106C000089B01A603B68002B5FD01D78324B1B683F
:106C1000002B04D05B68002B01D000209847260091
:106C200008363100E079FFF7B7FD237DE0710200FF
:106C3000E0780493638A29000393238A0293E3890B
:106C40000193A38800933300FFF752FFE378002BF2
:106C50000BD1E289A379A18802920196E2792800FA
:106C60000092012201F0DAFEE0703B68002B20D098
:106C7000FFF7ACFF194D287800281AD0184B197867
:106C8000FFF778FE002814D02B78E67808200793C9
:106C9000A78804F091FE011E09D0D0230370CA3BDF
:106CA0004670837087808671079804F07DFD00230D
:106CB0002B701721A088FFF775FCA08801F034FC29
:106CC000A08801F00BFD09B0F0BD064B9DE7C04662
:106CD0003409FF1FBC66FF1FD066FF1FB166FF1F90
:106CE000B066FF1F1445FF1FF8B5070008000E002F
:106CF00001F08AFE041E18D02620FFF78DFC051E29
:106D000000D12578062004F057FE041E0DD0002186
:106D1000062204F099FFD0232370C23B2100677044
:106D2000A370A680E8B204F03FFDF8BDF0B585B0D1
:106D300001930AAB1B78070002930BAB1B7808008A
:106D40000D000092039301F05FFE061E22D010207A
:106D500004F032FE041E1DD01022002104F074FF46
:106D60002620FFF759FC002800D13078D02323706B
:106D7000C13BA370009B21002372019B677063726B
:106D8000029BA580A372039BC0B2E3720C9BE360DD
:106D900004F00AFD05B0F0BDF7B50D00019001F05B
:106DA00033FE071E20D00E2004F006FE041E1BD06A
:106DB0002620FFF731FC061E00D13E78D023238029
:106DC000C53B0622A370F91DE01C04F055FF019B92
:106DD0002A0063810123DD401A401D4021002273F7
:106DE0006573F0B204F0E0FCF7BD0000F0B585B0CB
:106DF000029010000D0017000A9E039301F004FE9C
:106E0000041E31D0029B002B2ED1039B02795B071D
:106E100024D5122313430422002E08D10B990029F4
:106E200005D10C99002902D10D9900291AD01A43D5
:106E30000D9B2271002B00D0C9E0002E00D1CFE0C5
:106E4000002D00D0CCE0606A002801D004F0CCFC1A
:106E50001C21300004F040FF606205E002239A43E9
:106E60000E33D7E793432371654BBA00D458002CF7
:106E700000D1AAE0002E10D0236A002B03D11C20E1
:106E800004F0DAFC20625E4BBA00D358186A00287E
:106E900003D01C22310004F0EFFE0C9B002B12D01B
:106EA000574CBB001D596B6A002B03D1162004F010
:106EB000C3FC6862BB00E358586A002803D016225E
:106EC0000C9904F0D9FE0D9B002B11D04C4DBC0049
:106ED0006659B36A002B03D1142004F0ADFCB062F4
:106EE0002B59986A002803D014220D9904F0C4FE8F
:106EF000380001F089FD051E67D0414BBA00D35818
:106F0000002B62D01A6A3420002A00D11C389A6AF9
:106F1000002A01D0143080B20B9A002A01D01C3014
:106F200080B25B6A002B01D0163080B204F044FDC1
:106F3000041E4AD01822002104F086FE2620FFF706
:106F40006BFB0190002801D12B780193D023237093
:106F5000029B200063700A23294EA370039BBD008F
:106F6000A371AB59A780196A1830002905D01C22DB
:106F7000A06004F081FE200034307359996A002922
:106F800007D0030014221433E060029304F074FE6F
:106F900002980B9B002B08D003001C221C330B997A
:106FA0002061029304F068FE02987359596A00291F
:106FB00003D01622606104F05FFE6B462100187951
:106FC00004F0F2FB3800FFF7E3FC05B0F0BD10223F
:106FD0000D9B0D991B69A018236204F04DFE2CE750
:106FE0000B9B002B00D13FE7012D00D03CE7606AEE
:106FF000002801D004F0F8FB1C210B982AE7C046BA
:10700000B866FF1F10B5044C2068002803D004F0B8
:10701000EBFB0023236010BDAC66FF1F0B4B07B5D5
:107020001A68002A01D100200EBD6946531C0120B8
:1070300012780731FFF772FC0028F4D002780123A0
:10704000100018401A42EED0EEE7C046C866FF1F97
:10705000F0B51F4F01203B6887B0002B25D09B78EF
:10706000059300F0B3FB002821D00A20FFF7D4FAE3
:1070700004000B20FFF7D0FA164B05001E78731E94
:107080009E413B68F6B2191DD878FFF757FB3B6865
:107090002900DA7A043303929A79019302920090DC
:1070A00033002000059A04F01FFC07B0F0BDFFF785
:1070B000B5FF002805D00620FFF7AEFA0400072030
:1070C000D8E70820FFF7A8FA04000920D2E7C04655
:1070D000AC66FF1FA866FF1F70B50A4E0400337828
:1070E0000D00FF2B0DD0042004F066FC011E08D01B
:1070F000D0230370CE3B45708370C470307804F0A9
:1071000053FB70BD2445FF1F70B5040006200D0021
:1071100004F052FC011E0AD0D0230370CD3B8370D3
:10712000054B44701B688580187804F03DFB002CEB
:1071300001D0FFF767FF70BDAC66FF1FF8B5264FA3
:1071400006003B680D001124002B05D10522234BBE
:107150001B78134202D112242000F8BD204A1024CB
:107160001268002AF8D01278002AF5D0DB0719D56A
:107170002B789A1E012A1AD80C2004F05DFB1324E8
:1071800038600028E8D000230A22437029000670E6
:10719000023004F071FDFFF75BFF041E0AD0FFF719
:1071A00031FFD9E700F012FB0028E1D1E4E7002B22
:1071B000E2D0D0E70B4B1B78032BCDD11D20FFF77E
:1071C0002BFA094B18800028C6D0084B04211878E8
:1071D000074A04F089FDBFE7AC66FF1FA966FF1FE1
:1071E000C866FF1FA866FF1FA666FF1FD466FF1FA5
:1071F00060EA0000F7B50193194B14001A780523D3
:1072000006000F0012201A4221D0012920D1154B6F
:107210001D68002D1BD002201F2C18D8002C02D076
:10722000019B002B13D0104B1F221E706E1C0021DF
:10723000300004F009FD01992200300004F01CFD2B
:10724000310020002C70002F06D004F07DFDFEBD23
:10725000064B12201D68DCE704F0EEFCF7E7C046A1
:10726000A966FF1FC866FF1F2445FF1FC466FF1FD6
:10727000F8B50F4E12243368002B17D01B780F3C43
:10728000834213D100250B4F0221387804F0DCFB38
:10729000094B042138781D8004F0D6FB074B2800E9
:1072A0001D8033685C7004F0EFFA04002000F8BD24
:1072B000AC66FF1FD466FF1FC066FF1FA666FF1FD8
:1072C00070B5012823D11B4C2388002B03D01A4A08
:1072D0001578002D07D0194B1B68002B02D01878A9
:1072E000FFF7C6FF70BD3B2B02D93C3B2380F9E77B
:1072F000134E0221307804F0A7FBFA222388920073
:1073000002215A43307804F067FA2580EAE70B4BF4
:107310001B68002BE6D00B4B1B785B07E2D5084BB4
:107320000221187804F090FB0022024B1A80FFF72C
:1073300069FED7E7C066FF1FA466FF1FAC66FF1F8C
:10734000D466FF1FA966FF1FF8B51E4D28680028E8
:1073500003D004F049FA00232B601B4E306800284C
:1073600003D004F041FA00233360184F05243B7822
:1073700018002040234221D0154800F02BFA3B781A
:10738000234213D0202004F057FA2860002813D09D
:107390002022002104F058FC202004F04DFA041EA5
:1073A000306005D02022002104F04EFC002004E0D3
:1073B000286804F019FA2C601320F8BD00F00AFACE
:1073C000F4E7C046C866FF1FC466FF1FA966FF1F1B
:1073D0001845FF1F10B50A4C23681A1E0ED000284E
:1073E00008D10130587004F04FFA002805D0236806
:1073F000002B02D00021FFF787FE0122100010BDF4
:10740000AC66FF1FF7B5274E050033680191181EC3
:1074100021D05C78244F012C30D1FFF7FFFD0028EC
:1074200025D02000FFF7F8F80400412814D91F4B9D
:10743000022118781E4A04F057FC1E4B3C3C1C806D
:10744000022233685A703B78002B14D1280001992E
:10745000FFF75AFE0120FEBDFA2292004243002AA5
:10746000EED0124B0221187804F0B6F9E8E7FFF7E6
:10747000D3F80200F3E700233B70EBE73B78002BE7
:10748000E8D1032004F098FA011E08D0D02303703D
:10749000CC3B457083703368187804F085F9FFF7AA
:1074A000B1FDD7E7AC66FF1FA466FF1FD466FF1FC0
:1074B00060EA0000C066FF1F10B51749838802000C
:1074C0008B4220D011D815498B4217D01449002087
:1074D0005B1899B2012907D8926811785A42534132
:1074E000D8B2FFF7F9FD012010BD0E4A00209B180D
:1074F00007229BB29A424041C0B2F5E783681878F0
:10750000FFF768FFF0E7836899785A7809021878DE
:107510001143FFF777FFE7E70A200000062000008D
:10752000F8DFFFFFAFDFFFFF014B18707047C04669
:107530002545FF1F10B5064C207001F041FA207858
:1075400004F0FAF90521207800F062FD10BDC04674
:10755000D466FF1F0BB273B50D00002B00DBC4E037
:10756000884B187804F040FB041E0ED00378912B52
:107570000FD0A22B00D1A1E0834B1878FF2852D066
:10758000210004F011F900284DD18020000268404C
:1075900076BD43780F2B76D013D8052B70D00E2BE9
:1075A000EAD18088794B98422BD8794B98421BD8E6
:1075B000784B9842E0D1A3681878591CFFF774F80B
:1075C00038E03E2BD8D18378032B74D06CD8012BB4
:1075D0006ED0022BD0D1704B1B68002B23D05B6880
:1075E000002B20D098471EE06C4BC0180C28C3D845
:1075F00004F0BAF81DC2C2150BC20B0B0B3223C22A
:107600003C00674BC0180728B6D8664B1B68002B98
:1076100009D01B68002B06D0200098470AE0A36819
:107620001878FFF7C7F8200004F0B6F8ADE7A068B7
:10763000FFF762F800289FD0F5E7A3681B78002BBE
:10764000F1D0554B1B68002BEDD01B68002BEAD006
:10765000210055489847EDE74F4B1B68002BE2D0BF
:107660001B68002BDFD021005048F3E7504B1B680C
:10767000002BD8D05B68002BD5D021004348E9E728
:10768000FFF7EAF9CFE780884A4B984203D04A4B8C
:10769000984200D070E7464B1B68002BC3D05B6854
:1076A000002BC0D02100D5E7153B012BBBD963E7E8
:1076B000FFF798FAB7E7FFF77DFAB4E73F4B1B787F
:1076C000042B07D100236A4613800179408800F01B
:1076D000C5FCA8E7364B1B68002BA4D05B68002BC9
:1076E000A1D00100364898479DE7012421420AD0E5
:1076F000294B1B68002B04D05B68002B01D00020B5
:107700009847012043E78B070AD5264B1B68002BBF
:1077100004D05B68002B01D020009847022036E798
:107720000421280008400D4200D131E7254E33885E
:10773000002B21D0013B9BB23380002B1AD1FFF7E5
:10774000DBF800280AD0204B1C70164B1B68002B5E
:1077500004D05B68002B01D020009847FFF7C6F8E3
:10776000694601F001FD6846FEF7FEFF1D20FEF7A9
:1077700053FF308004200AE7024B187804F064F9C4
:10778000F8E7C046D466FF1F2545FF1F0E20000006
:107790000120000009100000CC66FF1FFEDFFFFF84
:1077A000AFDFFFFFD066FF1F0C2000000B200000A2
:1077B000B466FF1F0D20000013200000A966FF1F04
:1077C000FFFF0000A666FF1FA466FF1F10B501F0B3
:1077D0009BF910BD014B18607047C046D066FF1F73
:1077E0000B880020162B01D817230420014A138090
:1077F0007047C0467E66FF1F00207047074A03009F
:107800001188814207D091880020994202D101302D
:107810008000101870470020FAE7C046DC66FF1FA2
:10782000F0B58F7806000D00C7B01E2F15D1FFF7F9
:10783000E5FF051E03D10024200047B0F0BD002263
:107840003B003100C078009200F0B2FB0400A81C9D
:1078500000F0D3FBFF23EB70EEE7264B06240393E7
:107860001B78FF2BE8D0182FE6D87B08224A013B73
:10787000DB0002929A589446002ADDD0029AD3186F
:107880005B68002BD8D00878002802D14B78012BF8
:1078900002D10624122FCFD107AFAB8869780097A9
:1078A0006446AA68A047041EC6D1AB78029A5B085A
:1078B000013BDB00D318390030005B689847041E99
:1078C0000BD1AB78042BB6D0039A3100107822008C
:1078D000009700F06DFB0400AEE76A78002AABD198
:1078E000AA7805A93B88087130000A704B80FEF722
:1078F00047FBA0E72845FF1FB0BF00111D4B37B560
:10790000050098420BD000290AD1FFF777FF002825
:1079100005D11948FFF772FF002800D0058037BD58
:1079200001291AD1FFF76AFF041EF8D001235B4238
:107930000380A378FF2BF2D0FE2B07D00023E07842
:107940001422009329001E3300F032FBA01C00F02B
:1079500054FB01235B426380E1E70229DFD1013957
:1079600001F0BEF80028DAD12800FFF747FF041E17
:10797000DFD1D4E7FEFF0000FFFF0000022210B5B8
:10798000074B52421A80074801325A809A80DA80A7
:1079900000F07EFA044801F025F8002010BDC04632
:1079A000DC66FF1F21780011FD7800110388F7B510
:1079B0000400002B02D102252800FEBD42680221EE
:1079C000137825485268FEF7A5FD00282ED0234FD6
:1079D00001253A88002AEFD0802321885B02012507
:1079E0009B1A9942E8DC0C2003F026FF061E31D0DA
:1079F0003B8822889C4600231800019561469DB271
:107A0000491989B2AA421BD8002801D062443A80A1
:107A100000233000082208C0210004F02DF9104A8C
:107A20001368002B13D100251660C5E76268022198
:107A300013780C485268FEF76DFD0028C7D1BAE7ED
:107A400060681D014019418101330198D6E71A0091
:107A50001B68E6E71325AFE71EC000112645FF1F90
:107A6000D866FF1F1CC00011014B18707047C0463C
:107A70002845FF1F14230A0010B51A40194204D0EC
:107A80000122102101F048F810BD4B06F9D4012065
:107A900088434000F8E710B514008B0604D5012296
:107AA000102101F039F810BD08230A001A401942CC
:107AB00002D14BB2002B0FDA102101F02DF8002873
:107AC00008D02300F9331B78002BECD0F83423784E
:107AD000012BE8D10020E6E703208907FAD4E2E78A
:107AE000F0B51F00184B85B01C68019002910392FD
:107AF000002C27D1200005B0F0BDA5683301ED189A
:107B00006B89019A934211D3029A93420ED8002FA7
:107B100004D10A9B002B10D12C00EBE73B00297805
:107B2000039A6868FEF7F6FC0028F2D10136B6B277
:107B3000A388B342E1D82468DAE7A3680A9A5B898C
:107B40001380E9E70026F3E7D866FF1F37B50C007E
:107B50000A8849880123914217D3002A15D0651D50
:107B600023792A0002210A48FEF7D4FC10230028BA
:107B70000BD023796188208800242A000094FFF725
:107B8000AFFF0A23A04200D0230018003EBDC0462C
:107B90001EC0001113B50A000888498801238842D5
:107BA0000BD8002809D00024137905320094FFF780
:107BB00097FF0A23A04200D02300180016BD13B57A
:107BC0000A0008884988012388420BD8002809D078
:107BD0000024137905320094FFF782FF0A23A042A4
:107BE00000D02300180016BDF0B58BB003904A8872
:107BF00008880E000123824255D3002853D0002369
:107C0000012704AC23700022718813000092FFF753
:107C100067FF051E3ED02078002835D12B78022B37
:107C200018D167706A8983000130E31880005A8098
:107C300069680222201804F01FF823780133DBB2B0
:107C40002370042B19D93B006889013080B2002BC6
:107C5000D9D01FE002236370122358436A89231886
:107C600004305A8069681022201804F005F823783F
:107C70000133DBB22370002BE5D10C4A6B899B18D2
:107C80005A425341DBB2DFE76378012BE4D12B7812
:107C9000022BC7D022780A23002A04D0210003989F
:107CA000FEF798F9002318000BB0F0BD0100FFFFAC
:107CB0000F4BF0B504001868002816D083685D8962
:107CC000A54207D88288AE18B44203DA12019A1886
:107CD000934201D10068EFE71E005F891036A7428A
:107CE00004D1002900D00D801800F0BD3300EFE76B
:107CF000D866FF1F70B505000C0008880021FFF74B
:107D0000D7FF03000120002B04D022002800197A9D
:107D1000FFF7C1FE70BDF7B50C00002501902300F0
:107D2000F6331B78AB4201D800200AE06B00E65A1C
:107D300000213000E718FFF7BBFF002802D12680A2
:107D40000130FEBD017A0198FFF794FE002802D0B1
:107D50003B882380F5E70135EDB2E0E710B504007C
:107D600008880021FFF7A4FF03000120002B03D0A7
:107D70002000197AFFF77EFE10BD0000054B1B683E
:107D8000002B01D1180004E09A6852898242F6D192
:107D900098887047D866FF1FF0B50E27002687B079
:107DA000039302ABFF183E8005001F4B408914006F
:107DB000984207D02B78013000976A6880B2FFF7AD
:107DC0008FFE060002212B7818486A68FEF7A2FB96
:107DD00000280FD06C892000FFF7D0FF002802D0C8
:107DE000013C0419A4B2039B002B00D01C8030007E
:107DF00007B0F0BD02212B780D486A68FEF78AFBB8
:107E00000028E7D102212B780A486A68FEF782FB36
:107E1000002807D0002EDED03B88A342DBD1748936
:107E2000013CDFE76C89DEE7FFFF00001EC00011A8
:107E30001CC000111AC0001110B50C00FFF7DEFCC9
:107E400003000220002B0AD0002C00D023609B7876
:107E50001720FE2B03D00138FF2B00D1002010BDCE
:107E600073B50D0001A904001600FFF7E5FF172800
:107E700005D0002E04D129002000FEF727F976BD99
:107E800001221021200000F047FE0028F3D0F6E781
:107E9000014B18607047C046E866FF1F37B56B4658
:107EA0009D1D010004000222280003F035FE2B88EE
:107EB000B02B0ED12379122B09D12300FF339B78ED
:107EC000012B06D10121608800F0E0F801E01B2BB6
:107ED000F8D037BD10B5054B0421187000F098F8A4
:107EE000FFF74CFDFEF770FB10BDC046EC66FF1FB0
:107EF0000020F0B50BB20F0087B0834234DA274B75
:107F0000187803F071FE051E2BD00378A02B25D125
:107F100003AE3100FEF7E4F8041E0BD1B378DB07A3
:107F200024D51F4B06341B68002B03D03100688812
:107F300098470400A868002801D003F01DFC002C1D
:107F400008D1184A039B1340174A934206D0B378CE
:107F50001B2B03D00121688800F098F8280003F05B
:107F60001BFC80200002784007B0F0BD0F4B1B685F
:107F7000002B10D0310068889847041EDAD073783F
:107F8000002BD7D1B27801A90A704B800C71688898
:107F9000FDF7F6FFCEE70624F1E7C046EC66FF1FCB
:107FA000E466FF1F00FFFF0000011200E866FF1FEC
:107FB000F7B50190822040000D0017001E0003F06D
:107FC000FBFC04001320002C12D0B02320002370EF
:107FD000089BFC226770658026710830002B08D052
:107FE000190003F049FE2100019803F0DDFB002099
:107FF000FEBD089903F028FEF5E710B5041E06D073
:108000000078FD2803D803F007FCFF23237010BD80
:108010000A1F93B210B504000220032B05D882403A
:108020000020024BD1529B189C7010BD0C67FF1FA3
:108030000B8870B5043B04000D000220032B0BD805
:108040000121200000F04CFD03001420002B03D080
:108050002900200000F0DEFB70BD000007B5130012
:10806000034A00920A00012100F02CFC0EBDC0461C
:108070009982001107B5019203220092024B0A0077
:10808000122100F049FC0EBD1783001107B56B46A5
:1080900001AA11800449D88008780633012802D14A
:1080A000190003F0B9FD07BDED66FF1F0C4B10B5BD
:1080B00018700023FF210B4A138013819381938052
:1080C000094A53801370517293819372D174D38291
:1080D0001375517703F0F0FB00F0FCF910BDC046BA
:1080E0001C67FF1F0C67FF1FEE66FF1FF0B58DB00A
:1080F0006B46002003910C229B5E834200DBB0E0C4
:108100005D4B187803F070FD051E00D1A4E00378E4
:10811000902B00D09DE006AF01004688380000F0AB
:1081200013FA79680400002900D19CE03B88052BF4
:108130006ED13B89032B1CD905AC200000F0A2F8BE
:108140006288172A61D83989131D994231D179681B
:10815000237804310291D90738D5607800F08EF980
:10816000071E06D0002303712378012B08D0132BA0
:1081700023D0A868002800D178E003F0FDFA75E06C
:108180006288029909A800F0A6F80290380000F071
:108190008BF909AA2378387A0192002231000092E3
:1081A000029A00F012F9380000F064F9029B002BEB
:1081B000DFD0300000F080F9DBE70378032BD8D163
:1081C0006288029909A800F0D6F8DEE7122B13D1D5
:1081D000029909A800F0B5F8021EEAD127498B8858
:1081E000002BC6D0887909A9237801916178009184
:1081F000310000F0EAF8BCE7002302AA93833000C4
:10820000617809AAFFF72AFFB3E71D4B0993F6E748
:10821000042B02D09A1F012AABD8184A043B9B00BA
:10822000995A0029A5D0D218907831003A0000F070
:10823000AEF800289DD13B88042B03D001213000EB
:10824000FFF724FF012C04D1A868002801D003F017
:1082500093FA280003F0A0FA8020039B0002434019
:1082600018000DB0F0BD012800D182E701213000D7
:10827000FFF70CFFEDE7C0461C67FF1F0C67FF1FF1
:10828000010017000B7803704B784370CB788A7825
:108290001B021343438070470A88030002700A8858
:1082A000120A42700A88012A06D14A8882704A88D6
:1082B000120AC2700420704702208242FBD14A8811
:1082C00004309A704A88120ADA708A881A718A8889
:1082D000120A5A71EFE710B50400012082420CD94E
:1082E0004B780A781B0213432380834206D1CB7854
:1082F0008A781B0213436380002010BD022BFBD140
:10830000CB788A781B02134363804B790A791B026E
:108310001343A380F0E70B8803700B881B0A43709C
:108320004B8883704B881B0AC3708B8803718B88C2
:108330001B0A4371CB888371CB881B0AC371082049
:10834000704703000120082A14D14A7808781202E5
:1083500002431A80CA788878120202435A804A7906
:108360000879120202439A80CA798879120202437C
:108370000020DA80704710B504000120022A05D1E0
:1083800000204B780A781B021343238010BDF8B5F8
:10839000060010200F00150003F00EFB0400012062
:1083A000002C0ED0A0230C22290023806780201DE2
:1083B000002D07D003F060FC2100300003F0F4F939
:1083C0000020F8BD03F040FCF6E7F7B51E00009072
:1083D00008AB142017001D78019103F0EDFA041E7C
:1083E00012D0A2230370019B47704380099B057143
:1083F00046710C220830002B07D0190003F03CFC1A
:108400002100009803F0D0F9F7BD099903F01CFC96
:10841000F6E737B5041E0FD04388002B0CD000259B
:10842000C1881323007A172201950095FFF7CDFF2D
:10843000FF2365806372257037BD000010B50C49BD
:1084400004004A88002A09D08B89002B05D000201F
:10845000CB8A0222834201D010BD012213000A20E0
:10846000434300204032C854C81842800472F3E7E6
:10847000EE66FF1F0023438003707047094B002105
:108480001A0010B55C88002C06D01C79844203D1F8
:108490000A234B43D01810BD01310A330329F1D10F
:1084A0000020F8E7EE66FF1F10B50400407A03F0E5
:1084B000B3F9FF23637210BD7047043010B580B26A
:1084C00003F05AFA002803D00421494203F09CF932
:1084D00010BD000070B50025104CA0682580A58156
:1084E000A580A84202D003F047F9A56000250C4CF6
:1084F0000C4B606D1D80230058331D70A84202D0C4
:1085000003F03AF9656500256068002801D003F0A2
:1085100033F9013508340A2DF6D170BDB467FF1F59
:108520005867FF1FA867FF1F70B5041E09D1054DCE
:108530002880A881A880A868002802D003F01CF930
:10854000AC6070BDB467FF1FF0B54B8885B0019378
:10855000002343600A7905000F00022A00D07BE067
:10856000CA88032A17D98B685E7819783602DC78B6
:10857000D8790E4399781B7A24021B020C430343DB
:1085800053495BBA0B80331D93421ED1042C04D097
:10859000631F022B0ED9012015E0019A4D4B1201E9
:1085A000D35A002B06D00198FFF7BEFF4A4A136941
:1085B000013313610421B8682E812C80494203F0F5
:1085C00023F96860002005B0F0BD434D042C06D0AF
:1085D000631F022B0FD9EB680133EB60DBE7019AD5
:1085E0003C4B1201D35A002B05D00198FFF79CFF9A
:1085F0002B6901332B61374B30000293019B029AA8
:108600001B010193002301998C468B521300634494
:108610009C8003939E81FFF750FF039B041E98608C
:1086200016D00421B868494203F0EEF8FA88010038
:10863000043A200003F020FB0199029AFB888A5A31
:10864000043B9B18029A8B522B6801332B60A2E7E4
:10865000AB690133AB619EE71E4B0293019B1E0188
:10866000029BF35A002B2DD002998C19A068002888
:1086700028D0012A26D1FA889B189BB27352A1896F
:10868000994217D39B1AC018B96803F0F5FA029BF8
:10869000A289F35A934200D07DE700222B81A38860
:1086A0002B80A3686B60029BF2520B4A5368013324
:1086B000536070E7084A9368013393600198FFF7AD
:1086C00033FF68E7044A536901335361F6E7C04654
:1086D0001E67FF1FB467FF1F2467FF1F70B5051ECD
:1086E00015D10B4C0B4B1880230058331870606D5C
:1086F000002802D003F040F8656525005035606819
:10870000002801D003F038F80834AC42F7D170BD2E
:108710005867FF1FA867FF1FF0B51700A12285B09B
:10872000920001934243394B06001B680C009B18D2
:10873000D933FF331D78FDF741FF0430854204DD56
:108740003000FDF73BFF0430C5B2BD4207D33A000D
:1087500000213000019B03F017FB05B0F0BD29009C
:10876000380003F031F92300C6B250331E70039372
:10877000019B29006365380002F0BEFFCBB2029373
:10878000002B02D0039B01361E70002623005033BD
:1087900003931B78B34204D8606D002831D10020C8
:1087A000DBE7029A2800002A04D0013B1000B34204
:1087B00000D02800F700E719387003F0C5F9786099
:1087C00000280ED03A78019903F056FA019A3B78C6
:1087D0000136D3180E4A0193D369F6B20133D3613F
:1087E000D4E7039B18706065A74205D1084A13209F
:1087F000D36A0133D362B0E7606802F0BDFF08348A
:10880000F2E702F0B9FF00236365C8E73409FF1FF0
:108810002467FF1FF7B50D0007000421686802F008
:10882000F3FF2B89040003702B891B0A43702B88EC
:1088300083702B881B0AC3702E8902250436F6B27A
:10884000FB2E15D81B4B9F4214D10C2003F0B4F81B
:108850001135011E0CD0902303708E3B0371043B35
:108860004380154B8460C680187802F09DFF002578
:108870002800FEBD5C237B43104AD3180093583375
:1088800001931B78002B0FD10300320038000099B0
:10889000FFF742FF019B05001B78002BE8D1380051
:1088A000009903F029F9E3E7054A0725536A0133E4
:1088B0005362DDE7FEFF00001C67FF1F5867FF1FC4
:1088C0002467FF1FF0B587B0009017200F00160037
:1088D0000193FFF7F2FD1325041E19D00C98031E17
:1088E00002D00199201D9847030AE370052302AACC
:1088F000A0700430908127700098667003A993805F
:108900000494FFF787FF051E02D0200002F034FF19
:10891000280007B0F0BD0000F0B587B01F000CAB19
:108920001B780391059301210DAB06001C7804927E
:1089300000F0D6F81425002821D02000FFF77EFD96
:108940000135041E1BD01149059B0A7803700132C2
:10895000D2B2131EC68001D101231A000B702271FE
:108960003000049B03990097FFF7ACFF051E09D167
:10897000230021000648074A093303F0BDF9280007
:1089800007B0F0BD002363802370F8E72067FF1F66
:108990001384001130750000F8B505000E00064C78
:1089A000064F2368002B02D031002800984704347A
:1089B000BC42F6D1F8BDC046C467FF1FD867FF1F91
:1089C0000123064A5B425380002313715362044A19
:1089D000136053609360D36013617047D867FF1FC3
:1089E000C467FF1F0200002310B506499C00085908
:1089F000002801D1625010BD0133052BF6D11320A0
:108A0000F9E7C046C467FF1F034A5388181A434258
:108A10005841404210407047D867FF1FF0B585B0FD
:108A200002930AAB1F780CAB1B88009008000E0065
:108A300001920393FFF7E8FF05001120002D1BD1E1
:108A40000E48FFF7E1FF04001520002C14D0062289
:108A50000B99A771E01D03F00FF9019B3000237102
:108A6000029B29006371009B66802370039B6562F3
:108A7000E381FFF791FF280005B0F0BDFFFF000084
:108A800010B5FFF7C1FF04000220002C12D060884F
:108A90000121FFF781FF606A002801D002F0A4FEE7
:108AA00028220021200003F0CFF8012300205B42A0
:108AB0006380207110BD000030B5074A074C55880F
:108AC000010013780020A54204D05B1A59424B41A3
:108AD0005842104030BDC046D867FF1FFFFF00005E
:108AE000084A10B501230C00904208D0FFF78CFF14
:108AF000031E04D0037923405A1E9341DBB21800B1
:108B000010BDC046FEFF0000024B1879431E98417D
:108B1000C0B27047D867FF1F70B504000D00160083
:108B2000FFF772FF002804D10D4B9C4200D0143097
:108B300070BD416A03790520002907D012221A402E
:108B4000102A02D10520002EF2D10F20DB06EFD52E
:108B5000897E0C20A9428941494249420840E7E701
:108B6000FEFF0000030010B5002800D110BD03482F
:108B7000034A41889142F9D09847F7E7D867FF1F29
:108B8000FFFF0000002330B5C45CCD5C6C40D454C2
:108B90000133102BF8D130BD0F23002210B5C45C77
:108BA00064002243CA54C25CD209013BF7D210BD13
:108BB0000200010010B52032103102F02DFF10BD6F
:108BC000F0B58BB00390102005931700049102F0CC
:108BD00033FE0090102002F02FFE009B1324019022
:108BE000002B05D000280CD11324009802F0FCFDC6
:108BF000019B002B02D0180002F0F6FD20000BB004
:108C0000F0BD102002F018FE0600102002F014FE45
:108C100013240500002E00D1AEE0002819D0102248
:108C2000002103F011F832002900039802F0F4FE4D
:108C3000041E0ED133787F2B51D830000099FFF7F6
:108C4000ABFF009B1B787F2B53D801990098FFF74F
:108C5000A3FF300002F0C8FD002D02D0280002F072
:108C6000C3FD002CC1D1102002F0E6FD060010204B
:108C700002F0E2FD0290002E7CD0002878D03A006D
:108C80000F3223000125121105D00F333B4015B2DE
:108C90005A4253411BB26A1E1201002B33D0049B6F
:108CA000D2B298180099029AFFF76CFF013D10228A
:108CB0000021300002F0C8FFADB2049F2D017D19E4
:108CC000AF4242D0002C33D0300002F08DFD029B29
:108CD000002B00D189E7180002F086FD85E7290006
:108CE0003000FFF759FF28002549009AFFF74AFF97
:108CF000A7E729000098FFF74FFF28002049019AB5
:108D0000FFF740FFA5E70F210F4004998A18D9B259
:108D10008F4208D9D15C06A819540133102BF6D123
:108D2000029A0199C0E7791A48424141C901F2E724
:108D30003900300006AAFFF725FF3200039806A984
:108D400002F06AFE10370400BAE7002CBCD13000F4
:108D5000029906AAFFF716FF320006A9039802F04F
:108D60005BFE082204003100059802F085FFABE7A6
:108D70001324A9E71324AAE7002800D06EE733E7FD
:108D800024C00011F0B58BB00F0016000225009032
:108D900000283FD0002A3DD00B1DDBB21800029303
:108DA00002F04AFD1135041E34D0FDF747FD0500E1
:108DB0003A000099201D02F06FFDEBB20393E370BF
:108DC0002B0CDBB22F0A00936370FFB22B0E2370C3
:108DD000A7700193FDF72CFD1022010006A802F0F8
:108DE0005BFD2100029A04AB06A8FFF7E9FE051E11
:108DF0000DD1039B08223370009B04A9B370019B23
:108E00007770F370301D02F047FDFDF71DFD200067
:108E100002F0EAFC28000BB0F0BDF0B58FB00D00F9
:108E2000149E039004920593002A03D1022420008B
:108E30000FB0F0BD002EF9D00398FFF7E5FD142424
:108E4000071EF4D07278337812021A43B3781B04E9
:108E50001343F27812061A43036A0192934201D334
:108E60000133E3D1002D03D03B7901249B07DED5EC
:108E70000822002106A802F0E7FE059B1324043314
:108E8000DBB21800029302F0D7FC051ECFD0059A82
:108E90000499043002F000FD04223100280002F0A1
:108EA000FBFC3900102210310AA802F0F5FC290061
:108EB000029A06AB0AA8FFF783FE041E0FD1082210
:108EC00006A908A802F0E8FC0822311D08A802F053
:108ED0006BFE012807D101990398FDF7C9FC280012
:108EE00002F082FCA3E70124F9E7000070B51C4CF6
:108EF00005002368181E10D0002D14D11A78002AFE
:108F00000CD1981C083202F0B7FE02F045FE013584
:108F1000002808D123681D70012070BD0A33180095
:108F2000082202F0A9FE2368002BF5D0122002F0DF
:108F300043FD061E0DD0C123216803704570023128
:108F40001022023002F098FE23683100587802F0B7
:108F50002BFC206802F048FC00232360DCE7C046BD
:108F60000068FF1FF8B504002020FDF755FB0D4EEB
:108F7000A700BB590500002B0DD000280BD0D878D6
:108F8000FF2809D108492A000C55F3590748033333
:108F9000611802F0B1FEF8BD290002F06DFD002855
:108FA000F0D1F8E71C68FF1F0468FF1FBDA1001186
:108FB00070B5064D84006359002B05D0D87802F0B7
:108FC0002BFCFF226359DA7070BDC0461C68FF1F7E
:108FD00070B506008CB00C001500002130226846E8
:108FE00002F032FE31001022684602F055FC1D20CE
:108FF00021000322684402F04FFC6846FFF7D8FDC9
:109000002D21040003222800694402F045FC2000C1
:109010000CB070BDF0B50700160097B001931CAB03
:109020001D7830221EAB00910AA800211C7802F0A6
:109030000BFE102239000AA802F02EFC102200219B
:1090400002A802F001FE0722310002A802F024FC6F
:10905000072202AB9818631E9C41019902F01CFC88
:1090600002AB9C732B005A1E934102AAD3730021BA
:10907000102206A802F0E8FD06221D9907A802F0BA
:109080000BFC1A2002ABC01806221F9902F004FC48
:10909000102200990EA802F0FFFB102202AB0EA9CD
:1090A00008781C78013A6040D2B20870013301316F
:1090B000002AF5D10AA8FFF77BFD102212A90400AF
:1090C0000EA802F0D9FD102206AB0EA908781D7873
:1090D000013A6840D2B2087001330131002AF5D15B
:1090E0000AA8FFF765FD044310222098E4B212A9F4
:1090F00002F0D2FB200017B0F0BD70B50E001400D6
:109100008CB00100102268461D0002F0C5FB310042
:10911000082204A802F0C0FB2100082206A802F0E1
:10912000BBFB6846FFF744FD04001022280008A995
:1091300002F0B2FB20000CB070BDF8B506000D00C7
:1091400000243719AC4200D3F8BD02F06DFB030ACE
:109150003B70631CDBB201379D4203D90234F054EB
:10916000E4B2EEE71C00EDE773B506000C00022543
:10917000002819D0002917D0032101A8FFF7DDFF2F
:109180006B469A793F231A40013313436A463000F5
:10919000937101A92200FFF71BFF051E04D10322D2
:1091A000E01C01A902F068FD280076BD037858078D
:1091B000DA08C00FD20080009B0710439B0F1843B2
:1091C000C0B2704707230B40C908C9000B430370A6
:1091D0007047000070B50400FFF7EAFE134DA400CD
:1091E0006359002B21D0186A002801D002F0FCFA44
:1091F0002B59986E002801D002F0F6FA2B59D86E40
:10920000002801D002F0F0FA2B59186F002801D085
:1092100002F0EAFA2B59586F002801D002F0E4FA64
:10922000285902F0E1FA00232B5170BD1C68FF1F82
:109230000E4B8000C35870B50C00002B0FD09D68FA
:10924000002D0CD02B78201D0B706B784B70A97CF7
:10925000FFF7B8FF2B7E23726B69E36070BD1022AD
:109260000021200002F0F0FCF8E7C0461C68FF1F58
:10927000014B18607047C0461868FF1F074A03007B
:109280008000825810B5002A06D0D088984203D1B9
:10929000012901D1FFF79EFF10BDC0461C68FF1FCA
:1092A000F0B5264E95B087000B93BB590500099188
:1092B00012200A92002B31D0D888FFF7A5FB0400BA
:1092C0001420002C2AD0280010A9FFF7B1FFBB59A9
:1092D0001E781D6A002E23D00895FDF7EFFA0700CF
:1092E0000020FDF7F1FA0790A379E61D069310AD73
:1092F0000CA9089800F0E2FA0EA9280000F0D7FAAD
:109300000B9B0A990493069B09980293079B03966B
:10931000019300970EAB0CAAFFF77CFE15B0F0BDD1
:10932000FDF7CCFA06903000FDF7CEFAE31DA779E1
:10933000079310AB06000893DAE7C0461C68FF1FCE
:1093400030B50C4C85002A59030085B00120002A55
:109350000ED018006946FFF76BFF2B591A78D88892
:10936000054B002A00D1054B6A46072100F0D9FBC6
:1093700005B030BD1C68FF1FAF980011BD980011EB
:1093800030B5094C8500295985B010226846253131
:1093900002F072FC2A591121044BD0886A4600F071
:1093A000C0FB05B030BDC0461C68FF1F59990011B5
:1093B00030B5094C8500295985B0102268463531F1
:1093C00002F05AFC2A591121044BD0886A4600F059
:1093D000A8FB05B030BDC0461C68FF1F979900115F
:1093E000F7B54D4F86001020F4590D0002F024FA15
:1093F000F3592062186A132200286CD0033A29001E
:109400009C6802F039FCF3591A780192002A58D16D
:109410001E6A227D317B944651400122019F1142F8
:1094200001D167461740217D914339432175377B30
:109430004F40BC4660460027800701D44F081740C4
:10944000012102208F40227D82433A432275377BDF
:109450005740BC4660460027400701D497080F409C
:109460000420227DBF0082433A432275627D00279B
:1094700094466046727B42400A4201D167460F40E3
:109480000121627D8A433A436275777B5740BC462F
:1094900060460027800701D457080F400220627DF4
:1094A0007F00824317436775767B00227E407607F4
:1094B00001D4BA080A400426617D9200B1430A43F0
:1094C00062756A78002A08D06278002A05D00522E1
:1094D0000533DA7700221000FEBD042229791142FB
:1094E00005D1A17C114202D10533033AF1E7019A7B
:1094F00021782C78002A02D10A00210014001822B9
:109500000429E8D8042CE6D805206043034A053333
:109510001218525CDDE7C0461C68FF1F34C0001102
:1095200010B50A001121024B00F0FBFA10BDC04635
:10953000F39900110B0030B587B001AD2B806B465D
:1095400004001100981D082202F096FB2A000B214E
:109550002000024B00F0E5FA07B030BD1B9A001165
:1095600010B50A001121024B00F0DBFA10BDC04615
:109570006F9A001113B50B0011006A4613706B4609
:1095800004000622581C02F077FB6A4608212000DE
:10959000014B00F0C6FA13BD8F9A001110B50A00F6
:1095A0001121024B00F0BDFA10BDC046DF9A001138
:1095B0007FB505000B4BAA00D4580800002C0FD033
:1095C000666F237FE28821780396266F0296E66E07
:1095D0000196A46E0094FDF709FC2800FFF7FAFD40
:1095E0007FBDC0461C68FF1F10B51721FFF7E0FFC5
:1095F00010BD000070B50A000D00064B02210400EA
:1096000000F08FFA060029782000FFF7D1FF300024
:1096100070BDC046BF99001170B586B000236A4680
:109620001370836804001D78681E0A2859D801A9A0
:1096300002F0A2FA060633373B3F43474B4F530035
:10964000180000F042F9062312284BD000281BD145
:109650006088FFF7D9F90823002813D04279002A3F
:1096600047D1264B1A78072312070BD5244B1A68CB
:109670000723002A06D01668002E03D0290001AA6D
:10968000B04703006A4613706B461B786088002B56
:109690002AD1FFF767FC06B070BD180000F06CF926
:1096A000D4E7180000F087F9D0E7180000F093F92C
:1096B000CCE7180000F0ADF9C8E7180000F0C3F9D6
:1096C000C4E7180000F0F6F9C0E7180000F0F6F95A
:1096D000BCE7180000F013FAB8E7180000F013FA1E
:1096E000B4E707236A46137069466088FFF782FF74
:1096F000D1E70523012AC5D1024BB8E7A966FF1FB0
:109700001468FF1F1868FF1FF8B52C4F8600F35927
:1097100004000D00002B40D0DA8882423DD15A78F7
:10972000062A33D11A78002A2ED0012099681A6AA5
:10973000097D014206D0157B054203D007225A70ED
:109740000120F8BD0220014204D0157B054201D062
:109750000922F4E70420014204D0127B024201D026
:109760000B22ECE7164B1B68002BE9D05B68002B43
:10977000E6D020009847BB5900215B78122BDFD13F
:109780002000FFF715FFDBE70E4BECE7112A04D1B1
:10979000002900D032252900F2E7002D08D1200051
:1097A000FFF732F9002803D0102302791343037125
:1097B00021002800FDF798FAC2E7C0461C68FF1F89
:1097C0001468FF1F1868FF1F70B50E4E8500AB5957
:1097D0000400002B13D01B78002B11D10A4B1B68FF
:1097E000002B04D05B68002B01D0200098477359F0
:1097F0005B78122B03D100212000FFF7D9FE70BD4A
:10980000024BECE71C68FF1F1868FF1F1468FF1F5E
:10981000094B8000C3581020002B0CD01A6A002A74
:1098200009D09B68002B06D0127A1B7E101C9A422E
:1098300000D9181CC0B270471C68FF1F70B5030028
:109840000D0014000220002A30D000292ED0137001
:109850000B78081D53704B789370FFF7A7FCE070EE
:10986000012002212B7A23716B7B034063716A7B99
:109870000A401343042263716E7B164033436371C5
:109880006E7BF608F600334363712B7B0340A371B4
:10989000287B014000200B43A371297B0A4013431E
:1098A000A3712A7BD208D2001343A37170BD10B5F7
:1098B0000A0001000120FFF7C1FF10BD10B50A002A
:1098C00001000220FFF7BAFF10BD70B506000C00C2
:1098D0000220002E30D000292ED07378201D0B706E
:1098E000B3784B70F178FFF76DFC01223579257262
:1098F00071794B10080013409340104003438810C7
:1099000010408000C9080343C9000B436373B17959
:109910004B1008001340934010400343881002404E
:109920009200C9081343C9000B4321202373FCF79D
:1099300073FE854201D2122070BD2220257AFCF7E9
:109940006BFE8542F7D823781820042BF4D863786F
:10995000012BF1D80020EFE7030010B50220002909
:1099600009D0002B07D00322481C0A7019000D32C1
:1099700002F082F9002010BD03000222080010B599
:10998000002B06D0002904D00E32591C02F074F9C5
:109990000022100010BD030010B50220002909D0DC
:1099A000002B07D00422481C0A7019000C3202F068
:1099B00063F9002010BD10B5FFF7DEFF10BD0300F6
:1099C0000220002906D0002B04D0052200200A70B6
:1099D0001B784B70704703000220002B08D0002931
:1099E00006D05B7800200B70013B082B00D91830A3
:1099F0007047030010B50220002909D0002B07D0C2
:109A00000622481C0A7019000A3202F035F90020BB
:109A100010BD10B5FFF7B0FF10BD02000B00022013
:109A200010B500290ED0002A0CD00721197011881A
:109A300059701188090A997011180822D81C02F06F
:109A40001BF9002010BD03000A00022010B5002BF6
:109A50000CD000290AD09978587809020143118066
:109A6000901CD91C082202F007F9002010BD030049
:109A700010B50220002909D0002B07D00822481C6D
:109A80000A701900921802F0F7F8002010BD0200C9
:109A90000B00022010B500290BD0002A09D00921A3
:109AA0001970117818185970511C062202F0E4F848
:109AB000002010BD10B5FFF75FFF10BD02000B00C6
:109AC000022010B5002A09D0002907D0517819705A
:109AD00011180622581C02F0CFF8002010BD030018
:109AE00010B50220002909D0002B07D00A22481CFB
:109AF0000A701900063202F0BFF8002010BD10B540
:109B0000FFF73AFF10BD02000B00022010B5002A3B
:109B100006D0002904D018005178FFF753FB00202D
:109B200010BDF0B585B017001E006A46062305007B
:109B3000080091819380FEF7C0FC1324011E02905F
:109B40000CD03800B047041E05D1280001A9FEF74B
:109B50006FFA041E02D0029801F00EFE2800FFF7F3
:109B600001FA200005B0F0BDF0B504008BB0019102
:109B700015000021102202A802F066F8334EA7005B
:109B8000B85900283CD0C388A34239D10378002BB0
:109B900036D14278062A18D10200010055323531FB
:109BA0000C3006ABFFF7A9FA002829D12000FFF7F7
:109BB0002FFE020006A902A802F05EF8200002A90A
:109BC00001F01AFE01200BB0F0BD816E002917D004
:109BD0000B8A112A28D19D420ED101981231093ADF
:109BE00001F0E2FF012807D1BB5920009D6EFFF76D
:109BF0000FFE29000200DEE732212000FFF7D8FC2B
:109C00002000FEF701FF061E1BD0416A002918D074
:109C10000B8AAB4215D108220198123101F0C4FF22
:109C200001280ED1716A0AE09D42E9D1082201980B
:109C3000123101F0B9FF0128E2D1BB59996E8A7E39
:109C4000B9E7200001F070FDBCE7C0461C68FF1FAB
:109C5000F0B56B4D87007E5985B033780290039341
:109C6000002B00D087E0B368346A0193707806282F
:109C700017D101221B7D134202D0217B114218D142
:109C80000222134202D0217B114251D104221342FD
:109C900003D0237B134200D08BE0019B5A7DEB590C
:109CA00091E007380428F8D801F066FF032E4267D8
:109CB0008300B36E002B03D11C2001F0BDFDB06604
:109CC000EB599C6E002C1CD010220021200001F0CA
:109CD000BBFF0298FFF79CFD01002000FFF72DFA63
:109CE00001F0A2FD2082200008211230FFF725FAA2
:109CF0000298FFF78DFDA076EB592100D888FFF779
:109D00000FFC0822EB591CE0B36E002B05D01A00A3
:109D1000198AF0881232FFF70DFC0222019B197D8F
:109D2000EB5911423DD0207B10423AD0073208E077
:109D3000F488FCF7DBFD01002000FFF711FC0A228C
:109D4000EB595A70029B9C002A595378073B042B0D
:109D500011D8D088FEF758FE00284ED0C3895A0883
:109D6000D2182849029B0298CB542B59411804332E
:109D7000254801F0C1FF05B0F0BDFCF79FFD0300D1
:109D80000120834201D100200393EB59DE88FCF7C8
:109D90009BFD039902003000FFF7ECFB019AEB59A1
:109DA000117D042211420CD0217B114209D00B22DB
:109DB000C7E7F688FCF73CFD01003000FFF7EEFB3B
:109DC0006BE7019A527D01210A4204D0607B084270
:109DD00001D00C22B5E702210A4204D0607B084280
:109DE00001D00E22ADE704210A4204D0627B0A4270
:109DF00001D01022A5E71222A3E7FA225200B0E711
:109E00001C68FF1F2068FF1FC7A1001110B5064B7B
:109E10001A780423100018401A4200D00348FFF7B4
:109E200027FA002010BDC046A966FF1F2C45FF1F62
:109E300070B50400FFF7D4FA051E43D12000FFF7E8
:109E40007FFA234EA400A0598268937CDB0708D5D3
:109E50000321036A1B790B40012B02D1017F0B43C5
:109E60000377431DD97F8B1E022B0DD8022900D00A
:109E70000121C088FCF790FF042133591A7F5970E3
:109E80000A431A77280070BD01290CD10223102241
:109E9000437000210C3001F0D7FE305910213530CD
:109EA000FFF74BF9EEE70529ECD10223D1184370F7
:109EB00010220C3001F0E0FE04233259117F0B43D5
:109EC0001377EAE708251828DCD1053DDAE7C04614
:109ED0001C68FF1FF0B58BB0059143887E4F9E0034
:109EE000F45915000493002C15D1012902D000204B
:109EF0000BB0F0BD101D57781678FFF757F9EB68D7
:109F0000320002932B7A0499019300903B002000C9
:109F1000FCF70CFFEBE7E388049A934201D008209A
:109F2000E6E72378012B00D1D4E0059B581E0928D1
:109F300000D9CFE001F020FE05CE0A29CC506C8577
:109F40009AB229000498FFF773FFD1E72000290097
:109F50001022453001F090FEB9594B78042B02D104
:109F6000013B4B70C3E70B000A00253335320C313F
:109F70000498FFF795F90498FFF702FA0522431EAB
:109F80009841BB59C0005A70B2E720002900102246
:109F9000553001F071FE049B4F4C9D0029590498E7
:109FA0000A0006AB55320C31FFF77AF92959102215
:109FB000453106A801F0F8FD012808D10498FFF703
:109FC000F7F90590002804D106222B595A700598FC
:109FD0008EE708230593FAE763780C2B7AD1E36EBA
:109FE000002B03D11C2001F027FCE066BB59D86E82
:109FF00000286FD01022290001F03EFEBB590498C2
:10A00000DC6EFFF705FC0D22A076BB595A706EE797
:10A01000E06E00285ED063780D2B5BD12B88082280
:10A020000382A91C123001F027FEBB599A68517DAA
:10A030000222114226D0186A407B104222D00C32F4
:10A04000E4E763780E2B45D1236F002B03D1162054
:10A0500001F0F2FB2067BB59186F002803D01022D3
:10A06000290001F009FE0F22BB59CFE763780F2BBF
:10A0700030D1206F0622691C103001F0FDFDBB5964
:10A080009A68517D0422114203D0196A497B11421A
:10A09000D5D100210498FFF78BFA28E7636F002BD6
:10A0A0000DD0BB59586F0028F3D01022290001F0C1
:10A0B000E3FD0122BB5952425B6F1A61E9E71420AC
:10A0C00001F0BAFBBB5960675B6F002BE9D126E753
:10A0D0002978DFE707200BE71C68FF1F10B5064C47
:10A0E000207001F0D9FC06212078FDF791FF03488C
:10A0F000FEF778FC10BDC0462F68FF1F7D9200114F
:10A1000000200BB270B50D00834216DA264B18788A
:10A1100001F06AFD041E0DD00378922B0ED0A02B07
:10A1200037D0224B1878FF283AD0210001F03CFBB1
:10A13000002835D180200002684070BD43780E2B86
:10A140000BD03E2BEDD18378052B12D0082BE8D114
:10A1500081798088FFF7D8FA08E0154B82889A4207
:10A16000DFD183681878591CFEF7C0FE002817D18C
:10A17000D7E7104B1B785B0712D50F4B1B68002BE2
:10A180000ED09B68002B0BD0C289811D8088984718
:10A19000ECE7FFF741FAA068002801D001F0ECFAE3
:10A1A000200001F0F9FAC5E72F68FF1F2545FF1FC2
:10A1B00018200000A966FF1F1868FF1F10B500785F
:10A1C000FFF712FA10BD10B50078FFF7FDFA10BDC9
:10A1D0000C234343084A10B59B185A68002A03D041
:10A1E000012901D1904710BD9B68002BFBD00029AD
:10A1F000F9D19847F7E7C0464C68FF1F0123834019
:10A20000094A10B5946B1C439463506B9843506398
:10A21000D46B20009843012901D120001843D0635A
:10A22000116B0B43136310BD00800040F0B5002498
:10A230000127154B85B0DA6B144E03921A6C01920C
:10A24000DA64019BE3403B4217D0039DE5403D406B
:10A250000295E5B202992800FFF7BAFF316A736AE6
:10A26000002908D03900002B01D00299794028003C
:10A27000FFF7C4FF01E0002BF9D101340C36172C95
:10A28000DFD105B0F0BDC046008000403068FF1F40
:10A29000064B01215A68C2400A4204D01B68C340E1
:10A2A0001800084070471B6DF9E7C0460080004069
:10A2B0000122064B8240002903D0D9680A43DA60A4
:10A2C0007047D9689143D960FAE7C046003800402A
:10A2D00030B5032444430F4BE25C1B199C785D7836
:10A2E00001232D1B0135AB40013BA340A140DB43C3
:10A2F0000C00122807D8084992005218116819401A
:10A300002143116030BD054A11680B40234313609F
:10A31000F8E7C0467BC0001108F0004014F0004090
:10A32000C21F70B5D4B20623092C0BD80125084CE6
:10A330009540002908D00021FFF7CAFF23682B436E
:10A3400023600023180070BD2368AB43F8E7C046C4
:10A3500000380040214BF0B51B185B78022B21D14F
:10A36000032444431E4A1F4EA35C12199478012211
:10A3700015008540B76B013CE4B23D43A240B56394
:10A38000194C122815D89B0000290CD117495B18CD
:10A3900099680A439A600123205C154A834011683A
:10A3A0000B431360F0BD11495B18996891439960A4
:10A3B000F1E70E4B00290DD159690A435A61225C1D
:10A3C0001328E8D00123203A93400A490868034340
:10A3D0000B60E7E7596991435961F0E73068FF1F67
:10A3E0007BC0001100800040C0C0001100F00040A0
:10A3F000A0F00040A4F00040F8B500241B4E1C4D16
:10A400001C4B1B5D012B1FD1194A9269E2401A4275
:10A410000BD00122B25693402200143AD2B2022A43
:10A4200009D815494A6913434B61013402360C358A
:10A43000172CE5D1F8BD0022B2560F4992005218F0
:10A4400091680B439360F0E7022BEED1E7B238003E
:10A45000FFF71EFF01235840C1B23800FFF77AFF13
:10A460003800FFF715FF6877DFE7C0464DC00011E1
:10A470003068FF1F3168FF1F00F0004001220238E2
:10A480008240054B002903D059690A435A6170473D
:10A49000596991435961FAE700380040F8B50E0058
:10A4A00001210F008740114A0400D368FD43BB43DC
:10A4B000D360831E8B4201D8FFF7E0FF002120000C
:10A4C000FFF72EFF0A4A0B4B5168012E05D1394385
:10A4D0001B1951605E700020F8BD294051600222B6
:10A4E0001C1962709A6915409D61F4E700380040BC
:10A4F000008000403068FF1F012210B58240074BEA
:10A50000002906D019680A431A600121FFF7C6FF27
:10A5100010BD196891431960F7E7C04600800040FC
:10A520000C2370B5002543430A4A29009B181D706F
:10A53000094B04001B185D70FFF7B0FF0123A34017
:10A54000064928000A681A430A6005490A689A43BE
:10A550000A6070BD4C68FF1F3068FF1F34800040E8
:10A560003080004070B504000E00FF2813D0032592
:10A570000540FFF7D5FF084AA3089B009B183F2220
:10A58000ED00AA40AE4019682000914331431960A4
:10A590000121FFF78DFE70BD18380040F8B50C247E
:10A5A0004443134B0500E4186368002B03D1A368F0
:10A5B0001220002B1AD0022201270E4B00215B191A
:10A5C0005A7028002770FFF769FF63681E1E08D0C5
:10A5D000A3683E00002B04D02800FFF759FE464038
:10A5E000F6B228003100FFF709FE0020F8BDC04692
:10A5F0004C68FF1F3068FF1FF7B5C420FF222B4BAC
:10A6000080001958002491437F3A0A431A5080224F
:10A61000274F5202274E1A60274B1D5D002D21D077
:10A62000A31E012B03D80121E0B2FFF727FF012D64
:10A6300018D11F4B9B69E3402B4213D0E3B21800A3
:10A640000193FFF725FE01000198FFF755FFE3B2E4
:10A65000143B022B1DD801217156184A8D405369B5
:10A66000AB4353613B7F002B0DD0E5B22800FFF7D1
:10A6700095FF2800FFF70CFE7B7F0100834202D08C
:10A680002800FFF7A5FD01340C370236172CC3D183
:10A69000F7BD012100237156F3568D40074A9B00F8
:10A6A0009B189A68AA439A60DCE7C04600E100E084
:10A6B0003068FF1F4DC000113168FF1F00F00040DF
:10A6C00010B501210400FFF7E9FE0123044A002030
:10A6D00011194B70A34091690B43936110BDC046A3
:10A6E0003068FF1F70B50E0015000400FFF718FF5B
:10A6F0000C236343094A20009B189D605E60FFF7AE
:10A700004DFFF021064B074A8900051E5A5002D022
:10A710002000FFF705FF280070BDC0464C68FF1FF2
:10A720000000FF1F2DA2001170B5134D07202C78DB
:10A73000002C1FD1982221005200280001F08CFA31
:10A740000123C420FF222B700C4B80001C635C6330
:10A750000B4B1C605C600B4B195891437F3A0A43CA
:10A760001A50802252021A600D20074A074901F050
:10A770004BFA200070BDC0463068FF1F00800040CB
:10A78000A0F0004000E100E0F9A50011F9A30011DC
:10A79000030010B50620072B09D8054A137001F0F5
:10A7A0002BFAD7210020034B034A89005A5010BDD1
:10A7B0005445FF1F0000FF1F151BFF1F70B51D0034
:10A7C00002240C2910D8094ACA40D2070CD5FBF73D
:10A7D0002FFF041E08D1059A04992800FBF744FFB7
:10A7E000FCF7B2FDFFF712FB200070BD1210000055
:10A7F00030B50D7802232C009C43184201D02B4326
:10A800001C0008252300AB43284201D02B00234322
:10A8100020241D00A543204201D01C4325002A23EB
:10A820000D70184204D011781E3B0B43137030BDDD
:10A830000028FCD10C2113788B43F7E7F8B51D00F5
:10A8400006AB1B88140007AA0E000B201778002BFC
:10A8500027D10A78022A49D14A6850781178000233
:10A86000244A08438018042840D801F085F90312CF
:10A870001D1B2300F06801F0B7F8021CC0B2B842FB
:10A8800000D93A1CD2B22000F1682A8001F0F4F914
:10A8900006E00222F3681B882A8023701B0A63707B
:10A8A0000020F8BD0622EEE701232B80F3681B7819
:10A8B0002370F5E7F368002B16D008222A801A8847
:10A8C00022701A88120A62705A88A2705A88120A74
:10A8D000E2709A8822719A88120A6271DA88A271EB
:10A8E000DB881B0AE371DBE72B80D9E701202B8093
:10A8F000D7E7C04600D6FFFFF7B516000A781D005F
:10A9000008AB1F880C000123022A18D14A6850782E
:10A91000117800022B4A0843801803280FD801F051
:10A920002BF902254439E06801F05EF8C0B2072334
:10A93000B84204D37B190193152B02DD0D231800B7
:10A94000FEBDE0682A003100C01901F095F96B46A0
:10A9500000209B88E268D0541B4B1B68834203D0C5
:10A960001B68834200D098470023E8E70B23002FA1
:10A97000E5D1022DE2D1737832781B021343E268ED
:10A980001380114B1B68002BEED01B68002BEBD003
:10A990000120E8E70B23002FD1D1062DCED12A00CC
:10A9A0003100E06801F068F9DEE70B23002FC6D123
:10A9B000012DC3D132787533012AC0D8E3681A70EB
:10A9C000D2E7C04600D6FFFF3C6AFF1F70B50C00FF
:10A9D0001500072837D801F0CFF8041436361B3697
:10A9E000242E182015290BD8184E162200213000CD
:10A9F00001F02AF922002900300001F03DF9002081
:10AA000070BD18200229FBD11288114B1A80F6E77D
:10AA100018200829F4D10A000E48290001F07CF81A
:10AA2000EDE718200129EBD10B4B10780B49DA69BF
:10AA3000FFF7DEFEE3E718200129E1D1064B10788D
:10AA40000749DA6BF4E70220DAE7C046246AFF1F01
:10AA5000D245FF1FC845FF1F5845FF1F8045FF1FF8
:10AA6000A045FF1F030010B50020DB0704D5072118
:10AA7000024A034800F08CF810BDC046D8C000114F
:10AA80005845FF1F054A03001068002803D082883C
:10AA90009A4201D1806870470068F6E7406CFF1F5A
:10AAA0000A88030008009A4204D08A8804309A4237
:10AAB00000D0002070470000F8B5F82200230D4FA9
:10AAC0000D4E7968050042433370994200D07B6097
:10AAD0000A4C0021200001F0B7F800231A007C6026
:10AAE000AB4202D100203370F8BD01332280DBB2CB
:10AAF000F834F5E7406DFF1F3C6DFF1F446CFF1FEE
:10AB000073B56B4601900600684615001980FCF786
:10AB10004DFF041E11D1002D0FD07689002E11D0CB
:10AB20000C2000F089FE00280ED0084A046013684B
:10AB300086808560002B02D11060200076BD1A004F
:10AB40001B68F7E70224F8E71324F6E7406CFF1FC1
:10AB5000012100220A4B10B549420A4C1980998004
:10AB60009A719A70084B2070012019805A60FFF783
:10AB7000A3FF2078FCF778FF0448FDF733FF10BDF2
:10AB8000446AFF1F486DFF1F406DFF1F3DAC001161
:10AB9000022310B5002802D0FFF7B2FF030018000F
:10ABA00010BD0000030010B50020DB0704D5042110
:10ABB000024A0348FFF7A4FF10BDC046ECC00011D5
:10ABC000D845FF1FF0B50E2687B003930CAB1F8846
:10ABD00002ABF6180500080031000292FDF768F894
:10ABE00004000120002C0FD03088FFF74BFF03003A
:10ABF0000E20002B08D05E68002E05D02100280012
:10AC0000039B029A0097B04707B0F0BD0A4B10B5FE
:10AC1000984207D10122002352420A808B708A8019
:10AC20008B7110BDFFF73CFF0028FAD001235B4277
:10AC3000038000238370F4E7FFFF0000F8B50500F0
:10AC400001290AD1134E00243388F827AB4219D0CA
:10AC500028001149FFF7DAFF06E0022904D1013983
:10AC6000FDF73EFF0028EDD0F8BD3B00634372685E
:10AC7000D018D35A002B09D03A00002100F0E4FF8D
:10AC80000134E4B2054B1B78A342EED801235B42AA
:10AC90003380DDE7406DFF1F446AFF1F3C6DFF1FDF
:10ACA00010B5FFF7FDFE03000020834200D0987826
:10ACB00010BD0000F0B589B01C000EAB80CB039036
:10ACC0001E8810AB1B78049202930B7A0D00DB06F2
:10ACD00016D42B780593022B24D00498FFF7D2FECC
:10ACE000002812D003689C46002B0ED0029B220045
:10ACF000019329003B00644603980096A04705E0B5
:10AD00000498FFF7BFFE002802D10E2009B0F0BD65
:10AD10008368002BF9D00A2229000398984700285D
:10AD2000D7D0F3E76B6858781A786B4B0002104362
:10AD30009842D2D8043B984210D2684B984242D0F5
:10AD400015D8674BC0180128C7D80B20002EDDD1BD
:10AD5000EB681A7859683A80200028E0614BC018E7
:10AD6000032800D979E000F007FF846A789E5E4BE3
:10AD70009842B2D10B20002EC8D101233B80EB6852
:10AD800031001B7823706889013080B2FCF790FF96
:10AD90003A88031E0ED0017802328A183A8042891E
:10ADA00062704289120AA27059680278E01C00F0B1
:10ADB00063FF06E004323A8031000422601C00F098
:10ADC00043FF0020A2E70B20002E9FD1EB6807A9CC
:10ADD0001E8804233B80330A300026706370FCF722
:10ADE00067FF051E28D004AB9A890E2304A95B18BF
:10ADF0003E49C668FCF7D0FF00280BD12B783C48B1
:10AE00006A680599FBF786FB002803D1012304AA91
:10AE10005B42D3813278022A06D17168201D00F08E
:10AE20002BFF3B8802333B800E2304AA9B181B8810
:10AE3000A3701B0AE370C4E704ABDE81F4E70B20C8
:10AE4000002E00D062E7E9680398FFF729FF02238C
:10AE50003B802070000A6070B3E70B20002E00D00A
:10AE600054E70222EB681B883A8023701B0A637048
:10AE7000A7E7E86800F0B8FDC2B203000720B242BD
:10AE800000D243E70DD00299DBB27118994202DB80
:10AE9000921BD3B20293029BE9681A003B80891986
:10AEA0005AE70023F6E70B20002E00D02EE70722FA
:10AEB000EB683A801A7822705A7862705A88A270C9
:10AEC0005A88120AE2701A792271DA886271DB8874
:10AED0001B0AA37175E7C046042900000228000080
:10AEE00000D8FFFFFFD6FFFF03280000FFFF000090
:10AEF0001CC00011F0B58DB06B46002008912022D7
:10AF00009B5E83423DDAA64B187800F06DFE071E6B
:10AF100032D00378B02B2CD10079023816281FD8F4
:10AF200000F0D2FC17001E001E001E0031001E00A3
:10AF300096001E001D011E0052011E0073011E001E
:10AF4000CD011E0050021E001E001E008E021E00BB
:10AF5000E302944B94491B8878880B80FBF71AF81E
:10AF60003800FCF79BFF914B1B68002B01D0380089
:10AF70009847380000F010FC8020089B00024340F6
:10AF800018000DB0F0BDF6220021874800F05CFEED
:10AF90000BAA3B7B7989388900923A000D32FCF785
:10AFA0009FFD0400804B1B78002C3FD146E0804B76
:10AFB000788805937F4B4100CB5A0BAE073BDBB241
:10AFC00032880293002301937B4B21000693009368
:10AFD000059BFFF76FFE744D002810D1069B3A8A3F
:10AFE0001B889A420BD138000599123000F0DCFD25
:10AFF000002804D02B7862899B00EB185A80162316
:10B0000006A81B18328820007989FCF7C5FE2B782A
:10B0100004009A00AA1851880029C3D00133DBB27A
:10B020002B70002807D006A9C98A9180634A12882C
:10B030009A42BCD802E0012149429180002B04D001
:10B0400059497888FAF7DAFF8AE73E890A2479E0D5
:10B0500000253E89574B06937B88069A5B009B5AD6
:10B06000033B9D4202DB002DF0D05BE0162206A8D8
:10B0700012183B7B798900923A0030000D32FCF7C0
:10B080002FFD0590002858D04689017A7888FCF772
:10B09000F1FC041E44D1464B78880793069B41007F
:10B0A000C95A454B0439C9B206AAD28A06930291FD
:10B0B000019400930599079BFFF7FCFD041E2FD117
:10B0C000069B39491A88931C002D26D14B8079881C
:10B0D000384B4900CB5A5119033B8B4220DD059B6D
:10B0E00031485B8941190B71A91C0135C9B2EDB218
:10B0F000059145191B0A2B71059B2D49043318181E
:10B1000000F0BAFD2C4B059A1B88D318DDB22C4BEE
:10B110009E4205D00136B6B29CE749889942D6D006
:10B12000002D0CD0204C2800618800F0BDFC207060
:10B1300021007888FAF772FF12E7059CF0E7002CEF
:10B1400000D183E77B78142B00D109E716493B79BE
:10B150004E800B700C717888FAF712FF00E7162406
:10B1600006ABE41821003889FCF7A2FD011E00D1CE
:10B17000B7E1788822880F4C45002C5B0A4D013CD2
:10B18000E4B2029400240F4B01940095FFF792FD66
:10B19000041E00D014E129007888FAF74FFFDFE69B
:10B1A000486DFF1FC444FF1F4C6AFF1F406AFF1F0A
:10B1B000466BFF1F7C66FF1F3C6CFF1FC244FF1FD6
:10B1C000FFFF00004E6AFF1F162406ABE4182100A3
:10B1D0003889FCF76DFD011E00D182E17888228854
:10B1E000AE4C45002C5BAE4D013CE4B202947C8930
:10B1F000AC4B01940095FFF75DFD041E00D0DFE02D
:10B2000029007888FAF724FFAAE60025A44B1D80C0
:10B210003B00FE331B78A24A78880792AB4208D9DC
:10B220009E4B12880693069943005B5A013B9A4253
:10B2300003DB0799FAF716FF92E616246B00FB185A
:10B24000059306ABE418059B21001889FCF730FD37
:10B25000011E03D1059B01241E8973E77888924B58
:10B260002288069C099343001B5B904E013BDBB296
:10B270000293002300960193099BFFF71BFD041E18
:10B2800002D0059B1E895DE77B88069A5B009B5A6E
:10B29000079A108832881218934202DC1B1A013B6D
:10B2A00033807F4C023032880999001900F0E4FCA9
:10B2B0002388328801359B182380EDB2A8E70BAABA
:10B2C0003B7B7989388900923A000D32FCF708FC03
:10B2D00000250590059B002B04D10A24002D00D1E8
:10B2E0006EE060E0059B7888197AFCF7C3FB0100EB
:10B2F000041E63D1694C6C4B788806940993069BB5
:10B300004400E45A694B063CE4B20BAE3288079322
:10B310000294019100930599099BFFF7CBFC041E51
:10B320004CD1079B5E491B881A1D002D30D14A80E5
:10B33000059B5B4C5A8963191A716B1C9BB2E3180D
:10B34000120A1A71162306A832881B1879890598E3
:10B35000FCF722FDFF21AA1C2E1D03350B000590D2
:10B3600092B2B6B2ADB2002803D006ABDB8AD9B236
:10B370001B0AA218651911712B714C4D301D2A88BA
:10B380004949201800F078FC2B88F618B5B2A1E7DF
:10B390004988914207D17A8806995200525AEB188F
:10B3A000053A9A42C4DC3E4C2800618800F00CFB50
:10B3B000207021007888FAF75FFED1E5002DF2D1E8
:10B3C0003E89BFE6162606ABF61831003889FCF731
:10B3D0006FFC3D000400FF3500282DD0037A9B064A
:10B3E0000CD400227B893989788800923A000C328B
:10B3F000FFF7E8FB041E10D03E8915E03088FFF708
:10B4000041FB00281AD08368002B17D0210012229C
:10B4100078889847041EE4D0EEE7AB78002B02D181
:10B420007888FAF739FE0026AB78002B00D097E534
:10B43000002C00D194E585E60124DDE70E24DBE74E
:10B44000162506ABED1829003889FCF731FC041EDF
:10B4500047D0037A9B0611D4154A7B8811889942FC
:10B4600003D01448814207D11380134BF8261D786E
:10B470000023D9B2A94221D30924A1E72888FFF7E4
:10B4800001FB00282FD08368002B2CD02100122232
:10B4900078889847041EDFD092E7C0467C66FF1F7D
:10B4A0004C6AFF1F4E6AFF1F466BFF1F3C6CFF1F5D
:10B4B000406DFF1FFFFF00003C6DFF1F310059432F
:10B4C000546801336018615A0029D2D13C00083415
:10B4D0002100F82200F0D0FB21007888FAF7E4FD83
:10B4E0003EE501246CE70E246AE71D4B1A887B8831
:10B4F0009A4231D07888FAF7E1FD31E5F8230598D2
:10B5000051684343CD18C95A00291FD03B7A012BFB
:10B510000BD16C88AB887888AA1D0094FFF752FB8A
:10B52000041E02D000233B722E88F822002128003E
:10B5300000F08AFB00232B80059B0133DBB20593CF
:10B54000084B05991B78064A8B42D7D801235B42EA
:10B550001380002CCED0F5E5002634000596EFE7E9
:10B56000406DFF1F3C6DFF1F70B504000E001500FD
:10B57000FFF796FA031E08D131000548FFF790FA4D
:10B5800003001120002B02D01C8000209D7070BD94
:10B59000FFFF0000F8B50B4F06003B780D001400CC
:10B5A000FF2B0ED00A2000F007FA011E09D0B123AC
:10B5B0000380002346800371C5800481387800F041
:10B5C000F3F8F8BD1946FF1FF7B50F0008A90600EC
:10B5D000088809A90B240988002821D10234022BEC
:10B5E0001ED1557813782D021D432B008B430193F8
:10B5F0007334002B14D1FB68300019000093FFF75F
:10B600004FFB019C85420BD02A0030000099FFF7C8
:10B61000ABFF041E04D12A0030007989FFF7BAFF7E
:10B620002000FEBDF0B50E7885B003900AA805880D
:10B630000120022E0DD14C682778647824023C4307
:10B64000054FBC4205D10398DBB201960095FFF788
:10B65000BBFF05B0F0BDC0460229000010B50400D4
:10B660000C4800F069F80C48A16B00F065F80B4835
:10B67000E16B00F061F80A48216C00F05DF8094BBD
:10B680000948196800F058F8084B1B68002B00D0D7
:10B690009847FEE7CEBE0011E4BE0011F3BE0011D4
:10B6A00002BF001104ED00E011BF00114C6DFF1F3F
:10B6B000002307B501A80193FFF7D0FF044A05480E
:10B6C000002110B5121A00F0BFFAF8F773F9FEE77F
:10B6D000506DFF1F1C46FF1F01B40248844601BC89
:10B6E000604700BF6932FF1F01B40248844601BCB5
:10B6F000604700BFED4A010001B40248844601BC26
:10B70000604700BF090E000001B40248844601BC36
:10B71000604700BFC521000001B40248844601BC57
:10B72000604700BFC53F000001B40248844601BC29
:10B73000604700BF091B000001B40248844601BCF9
:10B74000604700BFE53A010001B40248844601BCED
:10B75000604700BF156B010001B40248844601BC7C
:10B76000604700BF2124000001B40248844601BCA8
:10B77000604700BFD13CFF1F01B40248844601BCB2
:10B78000604700BFD949010001B40248844601BCAA
:10B79000604700BFB537FF1F01B40248844601BCB3
:10B7A000604700BF434D010001B40248844601BC1C
:10B7B000604700BF594F010001B40248844601BCF4
:10B7C000604700BF6571010001B40248844601BCB6
:10B7D000604700BFC94A010001B40248844601BC69
:10B7E000604700BF8B52010001B40248844601BC8F
:10B7F000604700BF014C010001B40248844601BC0F
:10B80000604700BF311B000001B40248844601BC00
:10B81000604700BF5549010001B40248844601BC9D
:10B82000604700BF1147010001B40248844601BCD3
:10B83000604700BF2951010001B40248844601BCA1
:10B84000604700BF3D4B010001B40248844601BC83
:10B85000604700BF3D18000001B40248844601BCA7
:10B86000604700BF813AFF1F01B40248844601BC13
:10B87000604700BF75A9000001B40248844601BCBE
:10B88000604700BFC51D000001B40248844601BCEA
:10B89000604700BF691F000001B40248844601BC34
:10B8A000604700BF4551010001B40248844601BC15
:10B8B000604700BF3939FF1F01B40248844601BC0C
:10B8C000604700BF7918000001B40248844601BCFB
:10B8D000604700BFF93CFF1F01B40248844601BC29
:10B8E000604700BF413AFF1F01B40248844601BCD3
:10B8F000604700BF851F000001B40248844601BCB8
:10B90000604700BF8538FF1F01B40248844601BC70
:10B91000604700BF6DBC000001B40248844601BC12
:10B92000604700BF9137FF1F01B40248844601BC45
:10B93000604700BFDD66010001B40248844601BCD7
:10B94000604700BF5D17000001B40248844601BC97
:10B95000604700BF0124000001B40248844601BCD6
:10B96000604700BF056A000001B40248844601BC7C
:10B97000604700BFD53BFF1F01B40248844601BCAD
:10B98000604700BFE928000001B40248844601BCBA
:10B99000604700BF5125000001B40248844601BC45
:10B9A000604700BF4135FF1F01B40248844601BC17
:10B9B000604700BFADAE000001B40248844601BC40
:10B9C000604700BF1D4D010001B40248844601BC20
:10B9D000604700BF090E000001B40248844601BC64
:10B9E000604700BFEDA5000001B40248844601BCD9
:10B9F000604700BFDD52010001B40248844601BC2B
:10BA0000604700BFA54F010001B40248844601BC55
:10BA1000604700BFB54C010001B40248844601BC38
:10BA2000604700BFE548000001B40248844601BCFD
:10BA3000604700BFA93BFF1F01B40248844601BC18
:10BA4000604700BFDD30FF1F01B40248844601BCDF
:10BA5000604700BFB352010001B40248844601BCF4
:10BA6000604700BFA134FF1F01B40248844601BCF7
:10BA7000604700BF2526000001B40248844601BC8F
:10BA8000604700BF5147010001B40248844601BC31
:10BA9000604700BFC132FF1F01B40248844601BCA9
:10BAA000604700BFC926000001B40248844601BCBB
:10BAB000604700BF350E000001B40248844601BC57
:10BAC000604700BF093AFF1F01B40248844601BC29
:10BAD000604700BF350E000001B40248844601BC37
:10BAE000604700BF0189000001B40248844601BCE0
:10BAF000604700BF4550000001B40248844601BCC5
:10BB0000604700BF7D18FF1F01B40248844601BC96
:10BB1000604700BF0D52010001B40248844601BCD9
:10BB2000604700BF810E000001B40248844601BC9A
:10BB3000604700BF8132FF1F01B40248844601BC48
:10BB4000604700BF9130FF1F01B40248844601BC2A
:10BB5000604700BF017F000001B40248844601BC79
:10BB6000604700BFD1A5000001B40248844601BC73
:10BB7000604700BF3555000001B40248844601BC4F
:10BB8000604700BFE53CFF1F01B40248844601BC8A
:10BB9000604700BF3136FF1F01B40248844601BC34
:10BBA000604700BFD91B000001B40248844601BCB5
:10BBB000604700BFCD4C010001B40248844601BC7F
:10BBC000604700BFF539FF1F01B40248844601BC3D
:10BBD000604700BF2146010001B40248844601BC11
:10BBE000604700BFC95C010001B40248844601BC43
:10BBF000604700BFF54E010001B40248844601BC15
:10BC0000604700BF151BFF1F01B40248844601BCFA
:10BC1000604700BF0933FF1F01B40248844601BCDE
:10BC2000604700BFE117000001B40248844601BC30
:10BC3000604700BFB14E000001B40248844601BC19
:10BC4000604700BF5522000001B40248844601BC91
:10BC5000604700BF154D010001B40248844601BC95
:10BC6000604700BFB70E000001B40248844601BC23
:10BC7000604700BFC13AFF1F01B40248844601BCBF
:10BC8000604700BFE94C010001B40248844601BC92
:10BC9000604700BF055E000001B40248844601BC55
:10BCA000604700BF2D3BFF1F01B40248844601BC22
:10BCB000604700BFF30E000001B40248844601BC97
:10BCC000604700BF9DA9000001B40248844601BC42
:10BCD000604700BFC56D010001B40248844601BC45
:10BCE000604700BFF94C010001B40248844601BC22
:10BCF000604700BF5952010001B40248844601BCAC
:10BD0000604700BFA946010001B40248844601BC57
:10BD1000604700BF1D4B010001B40248844601BCCE
:10BD2000604700BF8D12000001B40248844601BC88
:10BD3000604700BF8552010001B40248844601BC3F
:10BD4000604700BFE134FF1F01B40248844601BCD4
:10BD5000604700BF4D1F000001B40248844601BC8B
:10BD6000604700BF456B010001B40248844601BC36
:10BD7000604700BFC9A9000001B40248844601BC65
:10BD8000604700BF291C000001B40248844601BC82
:08BD9000604700BF5118FF1FBE
:10BD9800000201030202030304030502060207026C
:10BDA800080209030A030B030C020D020E030F031A
:10BDB800100311031303140315001600913D00111D
:10BDC800C53D00110000000002000000DABD0011AE
:10BDD800192A0F180A000000F1590000FD2400007C
:10BDE80041460100ED80001101A1001155750011B7
:10BDF800F17E001159530011F5AE0011E54F001105
:10BE0800D93F00110941001100000000161600007A
:10BE18000200000024BE0011F4FFF3FFD2FC000072
:10BE2800D541001100000000000000005475796140
:10BE38000042312E31003030303100676974687546
:10BE4800622E636F6D2F7076767800544830350017
:10BE5800020000006CBE0011292A282A272A262A57
:10BE6800252A242A0A180000E204000071020000B2
:10BE780078EC0000744000001027000060F000001B
:10BE880006640000204E00000000000001000000D1
:10BE98001F501D00023CB4000001150011000000F5
:10BEA800A102000030313233343536373839414257
:10BEB80043444546005048592B36325858504C5543
:10BEC8005330353034005B48617264206661756CAC
:10BED800742068616E646C65725D0A004C522020A3
:10BEE800203D203078253038780A00504320202023
:10BEF8003D203078253038780A0050535220203DB4
:10BF0800203078253038780A0049435352203D20A4
:10BF18003078253038780A005D570011B157001184
:10BF2800000000000200000038BF00116F2A6E2ACE
:10BF38001A18EAC8BC80F0FC60FFFFFFFFFFFFFF94
:10BF4800FFFFF303B59747D6F613F7D777E6F0A7C1
:10BF5800F474000001A00000000000006410B71D88
:10BF6800C8206E3BAC30D9269041DC76F4516B6B1F
:10BF78005861B24D3C7105502083B8ED44930FF0E1
:10BF8800E8A3D6D68CB361CBB0C2649BD4D2D38697
:10BF980078E20AA01CF2BDBDFB349B5F80000080E4
:10BFA800001000000000000057610011E177001147
:10BFB8007B610011E97B0011FF610011BF7B00115B
:10BFC80075620011957B0011C76200115D7D00113B
:10BFD8002F6300115D7D001161630011177D001151
:10BFE800756200114D7B0011ED620011F57C0011A6
:10BFF8000000000000000000D3630011F57C001170
:10C0080035640011F9770011052A042A012A002A4B
:10C018000229032801280028011800180000000040
:10C02800000000000000000000000087010102017C
:10C0380002010102010203030401030101010101DC
:10C048000303020103000D000E001000110013008D
:10C058001401070108010A010B011C011D02040259
:10C0680005020702080219021A021C021D03010335
:10C07800020317000201000504000807000B0A006C
:10C088001716001D1C010201010504010E0D011106
:10C0980010011413011716011A19020201020B0AE2
:10C0A800020E0D02111002141302171603050403E1
:10C0B8000807030B0A030E0D0001020307090A0B08
:10C0C8000E0F101112141718191A1B1F2021220005
:10C0D8003DA80011F9A800110000000002000000AE
:10C0E80022C000110000000025B600110000000069
:08C0F8000200000020C000114D
:020000041FFFDC
:1000000000000000ED3E0011E0BD0011DCBD00115C
:100010002863FF1F00000000000000000000000037
:1000200000000000000000000000000000000000D0
:1000300000000000000000000000000000000000C0
:1000400000000000000000000000000000000000B0
:1000500000000000000000000000000000000000A0
:100060000000000000000000000000000000000090
:100070000000000000000000000000000000000080
:100080000000000000000000000000000000000070
:100090000000000000000000000000000000000060
:1000A0000000000000000000000000000000000050
:1000B0000000000000000000000000000000000040
:1000C0000000000000000000000000000000000030
:1000D0000000000000000000000000000000000020
:1000E0000000000000000000000000000000000010
:1000F0000000000000000000000000000000000000
:1001000000000000000000000000000000000000EF
:1001100000000000000000000000000000000000DF
:1001200000000000000000000000000000000000CF
:1001300000000000000000000000000000000000BF
:1001400000000000000000000000000000000000AF
:10015000000000000000000000000000000000009F
:10016000000000000000000000000000000000008F
:10017000000000000000000000000000000000007F
:10018000000000000000000000000000000000006F
:100190000535FF1F5533FF1FC16601000000000039
:1001A000000000000000000000000000000000004F
:1001B000000000000000000000000000000000003F
:1001C000000000000000000000000000000000002F
:1001D000000000000000000000000000000000001F
:1001E000000000000000000000000000000000000F
:1001F00000000000000000000000000000000000FF
:1002000000000000000000000000000000000000EE
:1002100000000000000000000000000000000000DE
:1002200000000000000000000000000000000000CE
:1002300000000000000000000000000000000000BE
:1002400000000000000000000000000000000000AE
:10025000000000000000000000000000000000009E
:10026000000000000000000000000000000000008E
:10027000000000000000000000000000000000007E
:10028000000000000000000000000000000000006E
:10029000000000000000000000000000000000005E
:1002A000000000000000000000000000000000004E
:1002B000000000000000000000000000000000003E
:1002C000000000000000000000000000000000002E
:1002D000000000000000000000000000000000001E
:1002E000000000000000000000000000000000000E
:1002F00000000000000000000000000000000000FE
:1003000000000000000000000000000000000000ED
:1003100000000000000000000000000000000000DD
:1003200000000000000000000000000000000000CD
:1003300000000000000000000000000000000000BD
:1003400000000000000000000000000000000000AD
:10035000000000000000000000000000000000009D
:10036000000000000000000000000000000000008D
:10037000B1B6001100000000000000000000000005
:10038000000000000000000000000000000000006D
:10039000000000000000000000000000000000005D
:1003A000000000000000000000000000951AFF1F80
:1003B000000000000000000000000000000000003D
:1003C000000000000000000000000000000000002D
:1003D000000000000000000000000000000000001D
:1003E000000000000000000000000000000000000D
:1003F00000000000000000000000000000000000FD
:081838005071FF1F4118FF1F52
:10184000024981F3088802F06BFC00005071FF1F11
:1018500010B502F055FC072804D0122808D0022841
:1018600008D010BD044A0420136B01331363F8E75A
:101870000220F6E71420F4E72467FF1FF8B50700FD
:101880000C0026002500503630785135002804D150
:101890000300287058342370F8BD2978CA00481E08
:1018A0008141A3183800A25C5B68C9B2FFF7D0FF82
:1018B00000280DD12B78DA00A218013350602B706C
:1018C0003378044A013B3370136A01331362D8E75B
:1018D0000123DFE72467FF1F5C234343074910B55B
:1018E000C9180B0058331B78012B05D1FFF7C6FF31
:1018F000034A936A0133936210BDC0465867FF1FC5
:101900002467FF1F10B502F0CBFB064A012113002C
:1019100010CB4942D967044B136002F031FB200021
:1019200010BDC04600E100E01000100010B504003A
:1019300002F0B6FB024B1C6002F022FB10BDC04659
:1019400000E100E010B5040002F0AAFB4021094AC2
:10195000200013688B43136002F0E2F901F0B4FD3C
:101960000022054B01201A60044B04321A6002F079
:1019700047FBFEE71CF00040C4F00040C0F0004010
:10198000431E5A425341A022F0B5D2015B4213409C
:10199000154D164A40019B182A18127E8BB00191F2
:1019A000002A1BD01A000832D46F0022E6B206AF1C
:1019B000E4B294420EDC2818C369002B08D00199C8
:1019C00002AA117106AA049202AA167303A89847E4
:1019D0000BB0F0BD1978B9540132EAE71A7D1A78D4
:1019E00006AB01261A70E6E7E469FF1F00400040DD
:1019F000F0B5254B04004001C25C85B0002A2BD015
:101A00001A18117E002927D0917E002924D011793F
:101A1000022921D11689D788D168F51BADB22A1CBD
:101A2000102D00D9102292B2BE4217D118180123EE
:101A300003710023C269C38003819A4206D06846BD
:101A4000032103730171029301A890470820002C21
:101A500000D0192001F034FC05B0F0BD013C654216
:101A60006C41A0256442ED012C40084D1B186419FF
:101A7000074D0633013A92B2AA42EDD01888461CAF
:101A80001E80085C2070F5E7E469FF1F00400040FD
:101A9000FFFF00000F220E4B10B59868104002386F
:101AA0000A280BD802F01EF90D0A0B0A0A110A0ABD
:101AB0000A0A060002210020FFF762FF10BD012183
:101AC000F9E70020FFF794FFF8E7DB6FF6E7C04681
:101AD000004000400F220E4B10B5986810400238AD
:101AE0000A280BD802F0FEF80E0A0B0A0A120A0A9C
:101AF0000A0A060002210120FFF742FF10BD012162
:101B00000800F9E70120FFF773FFF7E7DB6FF5E760
:101B10000090004013B5334C2378072B3DD8324B4F
:101B20001A78324B002A39D18022196852020A43AE
:101B30001A60252001F084FF20232D4A11680B43F1
:101B4000802113606B460422C905086807331042E0
:101B500028D080210422C905C86810422ED08021D7
:101B60002020C905CA688243CA6014221A701A78F4
:101B7000002A2FD18021C905C86820320243CA60DB
:101B800014221A701A78002A28D11A4B1A7D22784A
:101B90005A601D221A705932DA6013BD1A6816494C
:101BA0000A40C5E7086802430A6014221A701A78CE
:101BB000002ACED01A78013AD2B2F7E7C8680243B9
:101BC000CA6014221A7019784A1ED2B21A700029FB
:101BD000F9D1C4E71A78013AD2B2C7E71A78013AC4
:101BE000D2B2CEE75445FF1F1C46FF1F3CF0004019
:101BF0004C45FF1F00200040FFFFFEFF564B70B515
:101C00001B68012B03D1554A936D0133936502F094
:101C10008FFA534B534A1860534B544C1A600123AC
:101C2000534A1360534A13602378002B06D00622D0
:101C30005149524802F0C4F900232370504A514BD5
:101C400010681B78C1B2002B0ED14F4CC0B2237864
:101C50005BB2002B4FDB237824785BB264B21B04A9
:101C600024021B191B1813600B1C50294ED950233A
:101C7000464A47491078DBB2FF2202284BD1086858
:101C8000444C454D267890432A78964254D9227880
:101C900024782E78023B5D10A31B6B435201D31AAC
:101CA00010335B111843086002F032F9031F012B57
:101CB00045D83A4B1B78002B06D0394B1B78002BAC
:101CC00002D0002002F034F8A122364B920099781D
:101CD000354B4A431B689B18832292009B181B7844
:101CE000033B012B03D8AF20400002F059F9012239
:101CF0002E4BDA8270BD237824785BB264B2FF3356
:101D0000FF341B0424021B190138ABE7CAB2022AB4
:101D1000AED20223ACE70868254C264D26789043C6
:101D20002A78964208D9227824782D78023B5B10D5
:101D3000641B63435201B2E72378DBB2B2E70228A7
:101D4000D5D11D4B1B78013B022B03D91B4B1B78B4
:101D5000022BCCD16C20C8E79809FF1FFC0FFF1F96
:101D60005C66FF1FFF3F0000141003406066FF1F0A
:101D70000C10034000100340D50BFF1F7211FF1F12
:101D8000B40003408C09FF1F680AFF1F490AFF1FA8
:101D900094000340460AFF1F470AFF1FF908FF1F70
:101DA0002209FF1F300DFF1F3409FF1FBC0BFF1F4F
:101DB000440AFF1F450AFF1F1C09FF1F2309FF1FBD
:101DC00010B502F02DF80022014B1A8010BDC0465C
:101DD0005866FF1F10B502F09BF9A121054A890042
:101DE0009478054A61431268044B5218528C1A8049
:101DF00010BDC046300DFF1F3409FF1F5866FF1F7E
:101E000010B50D4B0D4A9978A1239B004B431268E6
:101E1000D218531DD97F0A4B1B88994209D2441C02
:101E200007D0C82805D0D2695B1A5A43054B5343E3
:101E3000C01802F005FA10BD300DFF1F3409FF1F56
:101E40005866FF1F7102000070B5244D2B68002BEF
:101E500028D002F0CDF82B68D8402B680400002B66
:101E600027D002F085F92B68D8401D4B1D4A997880
:101E7000A1239B004B431268D118D25C91239B0095
:101E8000002A20D0CA580132CA50174B17491B6884
:101E90000868834214D3D23B181A012A1AD0144B73
:101EA000186070BD02F0A4F8124B196802F0B8F87F
:101EB000D3E702F05DF90F4B196802F0B1F8D4E7EF
:101EC0000D495B18E8E7CA500C4B1B68DB68E41847
:101ED000201AE4E7F530FF30E1E7C0461C08FF1F99
:101EE000300DFF1F3409FF1F9C09FF1F5C66FF1F99
:101EF000A009FF1F1808FF1F2DFF3F006466FF1F8A
:101F000070B504000D00282916D10300A433C2883F
:101F10001B889B1A0B4A9BB293420DD906006A3666
:101F200005223100653002F05BF8002804D1310051
:101F3000200001F055FF70BD2900200001F0F8FFDE
:101F4000F9E7C046FE7F0000F8B50400012002F06A
:101F500097F801F0F5FF174A174910600968030068
:101F60001648174E01601748776805680020AF4291
:101F700001D27068281A144D091928601348C162EB
:101F8000A421446A49032143416211490978002987
:101F900005D010490978022902D10F3B1360F8BD22
:101FA000012901D1083BF9E7032901D1053BF5E7F8
:101FB000033BF3E7E408FF1F28F00040340AFF1F4B
:101FC00028100040180AFF1F1C0AFF1F00F00040E5
:101FD0001C09FF1F4A0AFF1F70B580241025E40565
:101FE000A3682B43A36001F0BBFFA368AB43A360CE
:101FF00070BD0000F7B5160080221C001023D2052A
:102000000191916805000B43936000225A4BD73031
:102010001A6002F01DF99D232A002F009B00EB5847
:10202000CA3201210092FC37002B01D00021009A16
:10203000386801F04DFF2900009BCB311A784F4BD7
:10204000D3351A604B780A781B0213438A7812043E
:102050001A43CB781B061343494A1BBA13604B79CA
:102060000A791B0213438A7912041A43CB7931008F
:102070001B061343434A1BBA13606B782A781B0272
:102080001343AA7812041A43EB781B0613433E4A03
:102090001BBA1360019A330213433C4A13603C4B52
:1020A00022001B1B9C4603293DDCB3089A00130049
:1020B0005142B21A032A46D1354AE018511A8278A1
:1020C0004078120400020243E05C043302430A60D9
:1020D0000022FF2B4BDDF0222E4B12011A600F2243
:1020E0002D4B1A602D4A1368002BFCD00023224A86
:1020F00027491360091B321D0B191B68043A180A83
:1021000023706070180C1B0EA070E3700434002A5A
:10211000F2DC802210213B68D20501333B609368DA
:102120008B439360F7BD6346D578981893782D0656
:102130001B042B43157804392B43557804322D02A8
:102140002B430360AFE7022A0AD1114AE05C511A1F
:10215000E2185278120202430A6004339BB2B7E7D6
:10216000012AB5D10A4A521AE15C1160F5E7084923
:1021700059180A600433ACE7000004403C000440F6
:102180003800044034000440300004400C00044097
:102190000001044004000440100004401400044006
:1021A000F7B5150080221C001023D205009191681C
:1021B00007000B4393600023654AD730136002F099
:1021C00047F89D233E009B00F9583B00CA36320079
:1021D000FC33002900D07FE0586801F079FE390017
:1021E00032785C4BCB311A604B780A781B02134370
:1021F0008A78AC4612041A43CB78281D1B06134379
:10220000554A1BBA13604B790A791B0213438A792A
:1022100012041A43CB791B061343504A1BBA1360AE
:102220004B7A0A7A1B0213438A7A12041A43CB7A36
:1022300021001B0613434A4A1BBA1360009A2B0263
:102240001343484A13602200474B1B1B0093009B1B
:10225000CE785B1801938B7836061B0433430E78D7
:10226000043833434E78043136023343019E3360E1
:102270000328ECDC0321A808431C9B0029408000B4
:1022800003292BD13849E5185E18A9786D78E35CED
:1022900009042D022943194331600300083300214A
:1022A000FF2B2DDD314B324919600F21314B196065
:1022B000012327490B60304B19680029FCD0062107
:1022C0001B680B40042B20D080220020D20593688D
:1022D0000A318B439360FEBD01217DE7022908D1BD
:1022E00021495D18E1184978E35C09021943296026
:1022F000D3E70129D3D11C495918E35C0B60CCE723
:102300001948181801600433CAE7002310490B600C
:102310006346002B0CDC3B00FC335A681021013271
:102320005A608022D205936801208B439360D2E7E4
:10233000009B9B181B68190A13705170190C1B0E17
:10234000D37004235B4291709C440432E0E7C046A2
:10235000000004403C0004403800044034000440C5
:10236000300004400C00044000010440040004401C
:10237000080F0000100004401400044070B5061E51
:1023800019D00222614B9B799343012B13D1604BEF
:102390001A78FF2A0FD15A78FF2A0CD19A78FF2A8F
:1023A00009D1DA78FF2A06D11A79FF2A03D15B799D
:1023B000FF2B00D1A7E0574B0C201A78012A08D038
:1023C0000022554D1A702B781A00093A042A01D8B8
:1023D000212070BD5A1F012AFAD94C4CA07B042839
:1023E00000D990E0A279032A00D98CE0821E012A4C
:1023F00003D862881F2A00D885E0002E61D0012E04
:1024000000D080E0A288012AE2D0002B0AD1013856
:10241000032803D801F066FC151D19151F202E7026
:1024200001F0F6FC2B785A1E032A16D800253B4BE8
:102430001D602823237501F02BFEA8422ED0A58015
:10244000C6E7022320202B70EAE7042322202B700A
:10245000E6E7032321202B70E2E7073B012BB7D8E7
:102460002F4B1B68DB6A9B06B2D52E4B1A78002ACD
:10247000AED1A27B911E012901D9002AA8D1022246
:1024800080211A702823284D89012878237501F0AE
:1024900027FE80212878890101F012FD0123A38005
:1024A000224B1B78002B0AD0FA228021204B92006D
:1024B0001B8809025A431C4B187801F0F9FD0020D3
:1024C00087E701F0EDFD2B78A680073B012B06D9AD
:1024D00018482E7001F08CFC1E2001F099FC114B65
:1024E000114C1A78002A06D0802100222078890118
:1024F0001A7001F0F5FD01F043FD802120780902FA
:1025000001F0EEFDDBE7122063E7C046A60BFF1FDC
:102510006B09FF1F1A09FF1F1C09FF1F4809FF1F36
:102520006466FF1F2309FF1F1B09FF1F2109FF1FEF
:102530002C09FF1F0010004010B5002901D001F048
:102540009FFC10BDF7B5604B01919978A1239B00CA
:102550004B435E4A060014681022E418D6235B0041
:10256000E0583623FF33E35C00279343222B41D10D
:10257000574B0F3A1A600760012501F029FD019BB6
:102580001880E8235B00E35C002B01D0B34258DDE8
:102590000023504FFB70AD33FF33E3581A68002A15
:1025A00003D09B88DB439B071DD03823FF33E35CBC
:1025B000002B18D09B235B00E35C002B13D1D1339D
:1025C000FF33E35CB3420EDAA4235B00E15AE01868
:1025D000090A023101F02CFE23000122FE33013EE4
:1025E00001351A87FA70E8235B00E35C002B2AD0E0
:1025F000A8B2FEBD03683D00002BBED08188043028
:10260000090A023101F014FED6235B00E3581F6073
:10261000B2E72300B133BA00FF33985801378188FD
:102620000430090A023101F003FEE8235B00E35C99
:10263000BB42EEDCE822F61AED1800235200A35448
:10264000A6E70027F1E7200001F002FD00281FD0D7
:10265000002E1DDD7319882647190193B60020004E
:1026600001F086FB5A3080002018406801358188CF
:102670000430090A023101F0DBFD200001F068FDA1
:10268000A3590133A351BD4202D0019B9D42E6D123
:10269000114BE35C002BABD095239B00E35C002B3C
:1026A000A6D00E4BE15A0029A2D00D4AA35C994254
:1026B00002D90133A3549BE700231A212000A3541D
:1026C00001F05EFB94E7C046300DFF1F3409FF1F89
:1026D00000140340E010FF1F5A02000072020000C5
:1026E0005E020000F8B51D4B1D4F1A78002A10D16C
:1026F000BA7B002A02D101321A7003E0032AFAD011
:10270000022AF8D001F0C4FC00220120154B1A70F7
:10271000F8BD154B154D1C68154B9E7801232B7089
:102720002878C0B200F0DEFCBB7B002B0BD101F09F
:10273000CFFCA1239B007343E41883239B00E41880
:1027400023782B70E4E7032B02D101F0A9FBF0E71B
:102750000020022BDCD101F033FDEAE71C09FF1F4A
:10276000A60BFF1F2309FF1F3409FF1F490AFF1F84
:10277000300DFF1FF0B587B00EAD2F780FAD2D785F
:102780000593AC46634614000E4D0CAA12782E78C1
:1027900003930D9B009201932200059B029701F089
:1027A00047FC2E70012C01D0042C08D18022064950
:1027B0008B889343054A1278D20113438B8007B06C
:1027C000F0BDC0461C09FF1F6C11FF1F7809FF1FD9
:1027D0000B001B3B70B504003020E02B0DD813001C
:1027E000E025493BFF3B9BB2ED00AB4205D8034BD4
:1027F000200019825A8201F0CBFA70BD8410FF1FAD
:1028000010B501F095FC054B00205B68052B04D941
:10281000034A5268D20200D4980810BD001000404C
:10282000FCE100E070B501F03BFC0D4B1B68FC3394
:10283000DC691D6AFFF7E4FF6419844204D2094B86
:1028400001241B68002B07D004220024064B1A70B9
:10285000064A93690133936101F092FB200070BD39
:102860006466FF1F9809FF1F2309FF1FFC0FFF1F4E
:1028700070B50C4D2B68FC335C6A01F011FCFFF75E
:10288000BFFF2B680025FC339B6AE318834204D208
:10289000054B1B68AB4200D1051B01F071FB280002
:1028A00070BDC0466466FF1F9809FF1FD722044B06
:1028B00092009B5810B5002B00D0984710BDC04621
:1028C0000000FF1FF0B587B001F096F9FFF7EEFFAB
:1028D000CA4BCB4C04931B78022B45D1C94B1B68C8
:1028E000186A01F0CDFBC84BC84A1A60C84BC94AE8
:1028F0001A60A022C84B52001A60049B187801F09D
:10290000EFFAC649C64801F0F3FAC649C64801F0D5
:10291000EFFA1022C54BFF201A60802252031A6082
:10292000802292031A60802212041A6001F000FAD9
:10293000012001F005FAFA20400001F0E1FA5820E8
:1029400001F02EFBBA4801F013FB012001F090FBCF
:10295000072001F0FDFA2268B64B1A4084235B0081
:102960001343236007B0F0BD01F04AFAB24E029063
:10297000322001F085FB33681B0629D43C2001F08E
:102980007FFB0F2001F07CFB9C4B1B78012B00D1BF
:102990001EE180223368A94D134200D0A7E02B68C6
:1029A000032013432B6001F06BFB01F029FA029B1B
:1029B0000299C31A5A1E814200D81A00A04B1A600D
:1029C000904B19681E2353439E4A9B18CB618AE79C
:1029D00001F016FA80239C4ADB02116803900B4336
:1029E00013602268934B994F1A40282313432360A6
:1029F000032001F045FB03203D6801F041FB3B68EB
:102A00000320DB03DB0B009301F03AFB3B68ED0393
:102A1000DB03ED0BDB0B8E4A0193AB18C22B30D8D6
:102A2000009B9B18C22B2CD8019B9B18C22B28D82B
:102A3000009B2A009D4200D21A00009B9D4200D9B3
:102A40001D00019B934200D21300019A954200D9C8
:102A500015005B1B122B14D80C22336814209343EF
:102A6000336033687B4A1340336001F009FB08216F
:102A70003B682268DB038A432260774ADB0B1360E2
:102A80007FE7032001F0FCFA3B68DB03DB0B0593D7
:102A900001F0B6F9039B0399C21A531E814200D874
:102AA00013006E4A93421BD9FF23356869492D0AEA
:102AB0001D4032686B1C1B060A401B0C134333601D
:102AC0000C23326800209A43083B1343336001F023
:102AD000AFF96348634BA840984206DCFEF732FF2B
:102AE000019B009D0093059B95E75F48F6E7002357
:102AF0005E4F554A3B6080231168DB020B43136035
:102B000080222B68032013432B6001F0B9FA3B6845
:102B1000052601333B6080232A685B0213432B6048
:102B20002268444B03201A40514B1343236001F0A9
:102B3000A7FA0821454B1A682368D2038B43236008
:102B4000454B023900931B68D20B4B439A420CD879
:102B50009B1A3B2B0BD8236846490B4023602B68FC
:102B60000B402B60444B1A601FE7D31AF1E7013E7C
:102B7000F6B2002ED4D123683E4A134023602B685E
:102B800013402B603B68042B07D9BFF34F8F3B4B9F
:102B90003B4ADA60BFF34F8FFEE780222B680320A9
:102BA00093432B6001F06CFA2268224B03201A40F9
:102BB00028231343236001F063FA244B009A1B6817
:102BC000DB03DB0B1360082223689343236097E742
:102BD00007222C4D2B681340012B02D1002001F05D
:102BE0007FF9AB68284A02201340AB6001F048FA35
:102BF0008023AA685B001343AB60D6E64A0AFF1F36
:102C00005CF000406466FF1F000003400180063D49
:102C1000BC00034034080000A4000340710200001F
:102C200014100040FFFF3F002810004000E100E0CA
:102C30003075000000FEFEFFC4F0004044F000408C
:102C40004C66FF1F7206000040F0004064F0004038
:102C500091FCFFFFFF00FFFF5466FF1FE30C000025
:102C6000E88000005F361E0060361E00B844FF1F7B
:102C700028000100FFFFFEFF5066FF1F00ED00E08F
:102C80000400FA053CF00040FFFEFFFF694E336888
:102C900088331B6883F3088801F09AF800F014FC6D
:102CA000654B664A1B68934207D0002001F0C0F8CC
:102CB0000221634A13688B431360FFF703FE614BE5
:102CC000614C1878C0B201F0ABFA0023A360023364
:102CD000A3605E4B0120236001F0D2F90323A360BF
:102CE00001F08EF8040001F023FA050001F088F8E5
:102CF000574B186001F054F8564B1968621A531E6E
:102D0000A14200D213008022D203934201D39B023E
:102D10009B0A3268D16AC90700D478E04E491C0C7E
:102D200009689BB24C4359432402090A64180327DB
:102D30004A49FC3293680A6849489B1A494A4A4EF4
:102D400012684A499B18414A34609A183B400193E3
:102D5000036892089C46019B0A6063440360042B4D
:102D600003D901323B400A6003600B684049E41814
:102D7000200001F055F93F4F3D493B68C3183B60C7
:102D80002000019301F06CF93B4C20680818384989
:102D90002060884205D9019B01333B6001F060F956
:102DA000216001F04DF8354B1B78002B0ED001F05F
:102DB000BFF93168324B4A1B1B6812189A4233D252
:102DC000591A4919091A2F4801F092F82E4C237A02
:102DD000002B0FD001F0ACF93168E3684A1B1218E0
:102DE000934224D9591A4919091A284801F080F840
:102DF00000232372264B83F3088801F0B1F90220E7
:102E000001F006F8002001F013F801F0C1F9DC012F
:102E100099000234641A5900641A09214B43803323
:102E2000CB40A408E41882E7FA218900CBE71949CE
:102E3000DBE7C0466466FF1F0C0AFF1FB641210393
:102E400010000040490AFF1F14100040C409000090
:102E5000100AFF1F340AFF1F380AFF1F200AFF1F36
:102E6000280AFF1F1C0AFF1F4866FF1F240AFF1FB6
:102E7000710200006008FF1F2C0AFF1F1C09FF1FC2
:102E8000E408FF1F00100040740BFF1F3C100040BF
:102E900000000020DC050000A022054B92009B589A
:102EA00010B5002B01D0984710BD01F0B1F8FBE739
:102EB0000000FF1FA122054B92009B5810B5002B6C
:102EC00001D0984710BD01F0A3F8FBE70000FF1FF9
:102ED000A222054B92009B5810B5002B01D09847B9
:102EE00010BD01F095F8FBE70000FF1FA322054B82
:102EF00092009B5810B5002B01D0984710BD01F0EF
:102F000087F8FBE70000FF1FA422054B92009B58A7
:102F100010B5002B01D0984710BD01F079F8FBE700
:102F20000000FF1F70B501F003F9514B1860042039
:102F300000F06EFF01F064F90400C30702D401F051
:102F40002FF970BD00224B4B1A604B4B187801389B
:102F500004282CD800F0C6FE03231B1F27002000E6
:102F600000F086FF0128ECD0444C2378042B71D16B
:102F700001F0BEF8002806D000F09AFF582001F0BA
:102F80000FF802232370032000F042FFD9E720004E
:102F900001F026F9E6E7200001F02AF9E2E7200037
:102FA00001F036F9DEE7200001F002F9DAE700F07F
:102FB000AFFF0500012808D1314B1B78053B012BE1
:102FC00003D82000FFF768FFCEE72C4B1B78022BBD
:102FD00001D0052B20D1022D28D12A4B9B7BAB435E
:102FE0001CD12000FFF766FF254B18780128BBD1C4
:102FF0006405B9D4234925224B7B034205D1233AEA
:1030000013405A42534126331A000B7D9342ABD9E9
:10301000322001F0DDF8A7E7022D07D1184B1B780D
:10302000052B11D12000FFF753FFDDE7012D0BD158
:10303000012B03D12000FFF759FF95E7062B03D1A1
:103040002000FFF761FF8FE7200000F0E1FF022D75
:103050008AD1C9E7032B04D10B4B987C00F000FF09
:1030600091E7072B8FD1094B987B00F091FF8AE7FE
:103070009C09FF1F9809FF1F9009FF1F2309FF1FCD
:103080001C09FF1FA60BFF1FBC0BFF1FD40BFF1F4C
:10309000FA210A4B0A4A49001A640A4A5A500A4A53
:1030A00004395A50094A08319A64094A5A50094A5F
:1030B0005C315A50084ADA667047C0460000FF1F6C
:1030C0007527FF1F7128FF1F2528FF1F7D23FF1F66
:1030D000E526FF1F011EFF1FD51DFF1F10B500F0C5
:1030E000E9FD10BD8023F7B59C46264B264F019382
:1030F0002649274A274D284C284B02281AD16046DA
:1031000038600868264E3040802636033043086019
:1031100001990978002909D11660224A2A60224AB9
:103120002260E02219689143A03A1BE08021C90285
:103130001160F2E766463E600F68194E3E408027F8
:10314000FF023E430E600199097800290DD11760F6
:1031500001280ED1154A2A60154A2260E02219681A
:103160009143C03A0A431A60F7BD80218902116079
:10317000EEE7E0210F4A02432A600F4A22601A68F4
:103180008A43F0E74B0AFF1FE0000340D8000340EA
:103190009000034000000340500003404000034003
:1031A000FFFFE3FF0280063D804508220180063DC7
:1031B000806608220080069880550822F8B51E4BCC
:1031C00080261A68002014003440324232D11A6836
:1031D0001A4F32431A6001223B68063093433B602A
:1031E00000F04EFF0122164D2B681E432E603B68F7
:1031F0000A2613433B608027BF00124B1B683B42EB
:1032000011D1013EF6B2FF2E09D17E220E4B1C6871
:103210002B68E40B1440934323432B6005E0082004
:1032200000F02EFFE9E7002EEFD180222B68600826
:1032300093432B60F8BDC046C4F000405CF00040F2
:1032400018F0004068F0004060F0004010B500F059
:1032500087FD01215820034A00F0F2FEFFF7AEFF80
:1032600010BDC046600AFF1F10B578220021034838
:1032700000F09EFE00F0ECFD002010BD6C69FF1F09
:1032800070B5040000F00CFF00230C200B4A010075
:1032900059438D18515C00290DD0A14208D101235A
:1032A00000246B7000F00CFF00F06AFE200070BD7F
:1032B00001330A2BEBD11224F6E7C0466C69FF1FDD
:1032C00070B5040000F0ECFE002319001D000D4A4B
:1032D0001078002806D0A0420CD1557001310C3274
:1032E0000A29F5D1002B0AD100F0B2FD00F048FE0A
:1032F000002070BD5078461EB0411B18EEE700F06C
:10330000DFFEF3E76C69FF1FF7B504000C20002314
:1033100084460E4D019267465F43E85D7E19A042E8
:1033200012D000280BD10A4B9C4662461B7808330A
:103330001370019B70707C557160B360FEBD0133EA
:103340000A2BE8D10320F9E70720F7E76C69FF1F94
:103350006869FF1F8021F8B5464BC9051B68C12469
:103360008B60454BFF261A68012313434B61434B87
:10337000A4001A68424B40201A60424B1A68424B24
:103380001A60424B1A59B2431A51C52292009D58F5
:10339000B5432843802598509F583D48ED0107408C
:1033A0003D439D509D5880272D022D0A2943995059
:1033B00080211A59090202400A431A5104341A5949
:1033C000344D3F042A403A4380271A511A593F0688
:1033D0001202120A3A431A5108341A5902400A4397
:1033E0001A51C32292009D58B5432C0080252C43CE
:1033F0009C509D582C0004400C439C509D58254CDB
:1034000025408024240425439D509C588025240277
:10341000240A3C439C50C424A4001A59B2432A43B2
:103420001A511A591202120A17431F5108341A5915
:10343000B24315431D5100251A5902400A431A513F
:1034400004341A59024011431951134C134B1B7881
:10345000DB08AB4201DC0020F8BD2378002B06D04E
:10346000A368002B00D0984701350C34EEE71220FA
:10347000F2E7C0465045FF1F4C45FF1FB0F000402B
:103480006469FF1FB4F000406069FF1F00E100E0C5
:10349000FF00FFFFFFFF00FF6C69FF1F6869FF1F50
:1034A000030010B51F2809D8072200201340072465
:1034B00004490A78A24313430B7010BD0023062071
:1034C000F5E7C0466869FF1F034A044913680020F6
:1034D0000B4013607047C0461CF00040FFFFC1FF67
:1034E000054B06491B780A6805485B0702401B0B21
:1034F000134300200B6070476869FF1F1CF00040F9
:10350000FFFFC1FF70B50C25FFF7EAFF0A4B1C78DF
:103510000A4BE4086543ED18002C01D1200070BD72
:103520002B78002B06D06B68002B00D09847013C0D
:103530000C3DF1E71220F2E76869FF1F6069FF1F89
:1035400007B50422074801A900F034F9019B0133B3
:1035500005D18023044ADB0411680B43136000206B
:103560000EBDC0461C18001114F00040F0B5050057
:103570002026184B87B00493049B002B03D1112401
:10358000200007B0F0BD002102220B000191009144
:10359000052000F0D5FD02230F490A681A42FCD12C
:1035A0000596059C631E0593002CFAD10B4A1368FF
:1035B000002BFCDA0F276F440121380000F0A8FB34
:1035C0003B782B42DCD0052000F05AFD049B013BE8
:1035D0000493D1E7FFFFFF0790C8004000C80040F8
:1035E00007B500F05DFD80220821D205936A0191A4
:1035F000002B01D10739916202210C4A1160019917
:10360000481E01900029FAD1033111600531019162
:103610000199481E01900029FAD11160002B02D1B6
:103620008022D205936200F0ABFC07BD00C00040D1
:10363000F0B52D4C89B02378002B4FD1FEF762F9FD
:1036400002232A4F03903A681A42FCD120230693A2
:10365000069B5A1E0692002BFAD1254E3368002B8A
:10366000FCDA0120FFF782FF011E02D0112009B011
:10367000F0BD030003220190009005AD9F2000F0F3
:103680005FFD0321280000F043FB02233A681A4241
:10369000FCD120230793079B5A1E0792002BFAD1D7
:1036A0003368002BFCDA0120FFF760FF0028DDD132
:1036B0000398FEF73BF9AA786B7811041B020B43C1
:1036C00029780B4363601300113B0A49052B07D887
:1036D00001239340A3600B60012323700020C6E701
:1036E00080231B03F6E7C0463845FF1F90C8004003
:1036F00000C800409808FF1F1E4B30B55A68187864
:103700001D4B85B0D31859424B4101210093002332
:1037100000F0BEFB194B1A4A02259A6300221A6573
:1037200010325A658022C4219D65164B1648D2027C
:10373000DA6789004258154B80241A4080231B0405
:1037400013434350642341200393E40500F078F9C8
:10375000402000F075F96562039D6B1E0393002DF8
:10376000FAD103236362FFF73BFFA562FFF760FF17
:1037700005B030BD4445FF1F95FFFEF700C800406F
:10378000050001FF04E100E000E100E0FFFF00FFB1
:1037900010B5064B18705960FFF7AEFF00211320DB
:1037A000034AFFF7B1FD002010BDC0464445FF1F8E
:1037B000F936FF1FF0B5040085B003920291FEF7C1
:1037C000A1F8882263035B0B52051A438023DB05B3
:1037D0009D6A8023274F0092BA68002601901B0340
:1037E0009A420CD9F82326001B041E401C4206D026
:1037F0008022214B52025E6219680A431A60002D32
:103800000BD100F04DFC02221C4B1A608023DB051B
:103810005A62013A9A6200F0B3FB0023039A934282
:1038200020D1002D0AD100F03BFC144B03221D6077
:103830008023DB055A629D6200F0A2FB8023BA68F8
:103840001B039A4208D9002E06D000220A4B0C49CD
:103850005A621A680A401A600198FEF767F8002059
:1038600005B0F0BD009A0299D2181278CA540133FB
:10387000D4E7C0463845FF1F00C8004000C00040E4
:10388000FFFFFEFFF0B587B0029103920400FEF740
:1038900039F8019000F004FC802302250122234E18
:1038A000DB0535605D629A6200F06AFB204F3B6881
:1038B0002B42FCD120230493049B5A1E0492002B1C
:1038C000FAD11C4D2B68002BFCDA0120FFF74EFECD
:1038D000002802D0112007B0F0BD2000039A029901
:1038E00000F01EFB022304003A681A42FCD1202398
:1038F0000593059B5A1E0592002BFAD12B68002BCD
:10390000FCDA0120FFF732FE051EE3D100F0C8FB10
:1039100080230322DB0535605A629D6200F030FB94
:103920000198FEF703F8E0B2D5E7C04600C00040BA
:1039300090C8004000C80040F0B5802687B0040061
:10394000FDF7E0FFF605B36A02250393029000F04D
:10395000A7FB0123244F3D607562B36200F010FBAA
:10396000224E33682B42FCD120230493049B5A1E21
:103970000492002BFAD11E4D2B68002BFCDA01209B
:10398000FFF7F4FD002802D0112007B0F0BD2000A1
:1039900000F00EFA0223019032681A42FCD1202373
:1039A0000593059B5A1E0592002BFAD12B68002B1C
:1039B000FCDA0320FFF7DAFD041EE5D100F070FB0E
:1039C00080230322DB053C605A629C6200F0D8FA37
:1039D000039B002B01D1FFF703FE0298FDF7A6FF22
:1039E0006B461879D1E7C04600C0004090C800403F
:1039F00000C8004007B5000201910422000A01A995
:103A0000FFF740FF0EBD000073B5050005240B4A0B
:103A1000A3005B429B1819686B46DE1D300000F066
:103A2000AFFB022804D133782B55013CEFD276BD91
:103A3000052CFCD00128FAD10230F8E71409001156
:103A40001F2807D8012380228340D20591680B43A9
:103A5000936070473F2808D8012380222038834094
:103A6000D20551690B435361F3E75F28F1D8012375
:103A7000802240388340D205116A0B431362E8E785
:103A80001F2807D8012280218240C9058B689343F3
:103A90008B6070473F2808D801228021203882405F
:103AA000C9054B6993434B61F3E75F28F1D80122C5
:103AB000802140388240C9050B6A93430B62E8E7D6
:103AC0001F2810D880230200DB05153A1968012A47
:103AD00006D820229143196019680A431A6070477A
:103AE00001228240F6E73F2811D880230200DB053F
:103AF000353AD968032A06D810229143D960D9688B
:103B00000A43DA60EBE7012220388240F5E75F28BC
:103B1000E5D842238022181A413B8340D205516ADE
:103B200099435162516A0B435362D8E710B50400C0
:103B3000012813D1A022184992050B685B015B098B
:103B400013430B60154B164A19681140154A0A4376
:103B50001A60402219680A431A6010BD0028FCD17F
:103B600001000A2000F02CF921000B2000F028F9B8
:103B7000C0220A4B920019680A4340211A601A6851
:103B80008A431A60B022044912060B685B015B0984
:103B900013430B60E1E7C04614F000401CF0004006
:103BA0007F00FEFF80FD010072B6074A13680133F3
:103BB00013600422054B1A600023054A136080221B
:103BC000D2055360FEE7C0467808FF1FC0F00040F2
:103BD000C4F00040044B054A1A60054B1A600022ED
:103BE000044B1A607047C046140AFF1F841E000071
:103BF000380AFF1FC4F000400023034A1360034A41
:103C00001360034A1360704754F0004040F10040D5
:103C100044F10040002310B5184C8AB00093019382
:103C20002378012B27D06946012000F091F8002865
:103C300017D1009B12490293019B06AA0393114BD3
:103C400002A81B680493104B1B68059300F088F9C9
:103C500010220E4906A800F0C3F9002804D1FF2362
:103C6000237000200AB010BD0123094A074902A8A9
:103C7000237000F075F90120F4E7C0466866FF1F65
:103C800010290011082900110C2900112029001108
:103C90006C66FF1F13B501246946012000F058F837
:103CA000034B00940193FFF7B5FF200016BDC046FB
:103CB000BB0B000010B5FFF79FFFFFF7EBFF0028DD
:103CC00002D0024B984710BDFEE7C046E1A20000BB
:103CD00002B4714649084900095649008E4402BCA5
:103CE0007047C04602B4714649084900095C490062
:103CF0008E4402BC7047C04603B471464908400078
:103D00004900095A49008E4403BC70470000000076
:103D100001B40248844601BC604700BF3D71010008
:103D200001B40248844601BC604700BFF9A6000008
:103D300001B40248844601BC604700BFED6B01003E
:103D400001B40248844601BC604700BF691101000C
:103D500001B40248844601BC604700BFE1AC0000EA
:103D600001B40248844601BC604700BFED68010011
:103D700001B40248844601BC604700BFD9B00000CE
:103D800001B40248844601BC604700BF53B900003B
:103D900001B40248844601BC604700BF116E0000B8
:103DA00001B40248844601BC604700BFC1660100FF
:103DB00001B40248844601BC604700BFA96F0100FE
:103DC00001B40248844601BC604700BFD1A2001183
:103DD00001B40248844601BC604700BFC9A9000085
:103DE00001B40248844601BC604700BF85C10000A1
:103DF00001B40248844601BC604700BFC1A5000071
:103E000001B40248844601BC604700BF156B010045
:103E100001B40248844601BC604700BF1907010095
:103E200001B40248844601BC604700BF8D82000097
:103E300001B40248844601BC604700BF016C010028
:103E400001B40248844601BC604700BFD54401006C
:103E500001B40248844601BC604700BFADAE00001B
:103E600001B40248844601BC604700BF4DF9000020
:103E700001B40248844601BC604700BF0134010020
:103E800001B40248844601BC604700BFE9D4000089
:103E900001B40248844601BC604700BFC56D010003
:103EA00001B40248844601BC604700BF75F80000B9
:103EB00001B40248844601BC604700BF6DF60000B3
:103EC00001B40248844601BC604700BF0D520100A6
:103ED00001B40248844601BC604700BF2144000091
:103EE00001B40248844601BC604700BFEDA5000054
:103EF00001B40248844601BC604700BF2D6C01003C
:103F000001B40248844601BC604700BF851201002D
:103F100001B40248844601BC604700BFDD0C0100CB
:103F200001B40248844601BC604700BF957301009C
:103F300001B40248844601BC604700BF51B800008C
:103F400001B40248844601BC604700BFBD5C01006B
:103F500001B40248844601BC604700BFF90D01006E
:103F600001B40248844601BC604700BFDD3F000049
:103F700001B40248844601BC604700BF8D110100B6
:103F800001B40248844601BC604700BF9DA90000FF
:103F900001B40248844601BC604700BFC1F700007D
:103FA00001B40248844601BC604700BF7912010099
:103FB00001B40248844601BC604700BFB70E000050
:103FC00001B40248844601BC604700BFE94C0100CF
:103FD00001B40248844601BC604700BFCD0C01001B
:103FE00001B40248844601BC604700BFCD4C0100CB
:103FF00001B40248844601BC604700BFE90B0100E0
:1040000001B40248844601BC604700BFA1AF000074
:1040100001B40248844601BC604700BFE9170100B3
:1040200001B40248844601BC604700BF090E00008D
:1040300001B40248844601BC604700BF9D6A00008D
:1040400001B40248844601BC604700BF016701001B
:1040500001B40248844601BC604700BF71B0000053
:1040600001B40248844601BC604700BF090E00004D
:1040700001B40248844601BC604700BFE51201005C
:1040800001B40248844601BC604700BF01890000BA
:1040900001B40248844601BC604700BFA9D80000B3
:1040A00001B40248844601BC604700BF75A9000006
:1040B00001B40248844601BC604700BF8B52010036
:1040C00001B40248844601BC604700BF21A900003A
:1040D00001B40248844601BC604700BFE9F6000015
:1040E00001B40248844601BC604700BFB3520100DE
:1040F00001B40248844601BC604700BF01D70000FC
:1041000001B40248844601BC604700BFE9270000B3
:1041100001B40248844601BC604700BFF9ED0000CD
:1041200001B40248844601BC604700BFBDB600111F
:1041300001B40248844601BC604700BFC95C01006D
:1041400001B40248844601BC604700BF496D0100CC
:1041500001B40248844601BC604700BF59760100A3
:1041600001B40248844601BC604700BF7997000053
:1041700001B40248844601BC604700BF6D0B0100DA
:1041800001B40248844601BC604700BF8D3800116D
:1041900001B40248844601BC604700BF855201005B
:1041A00001B40248844601BC604700BFDD0A01003B
:1041B00001B40248844601BC604700BFF9350100E4
:1041C00001B40248844601BC604700BF19FA0000F0
:1041D00001B40248844601BC604700BF613701005A
:1041E00001B40248844601BC604700BF09340100A5
:1041F00001B40248844601BC604700BF0534010099
:1042000001B40248844601BC604700BFBD0B0100F9
:1042100001B40248844601BC604700BFF535010087
:1042200001B40248844601BC604700BF8914010004
:1042300001B40248844601BC604700BFC1150100BB
:1042400001B40248844601BC604700BF89370100C1
:1042500001B40248844601BC604700BF89440000A5
:10426000020000001EC0001101000000D0BD0011BE
:10427000020000001AC0001101000000A042FF1F50
:1042800002000000D8BD001101000000A863FF1F5C
:104290000200000018C00011030000001C63FF1F93
:1042A00012000000020000001EC00011010000000A
:1042B00018BE0011020000001AC000110100000029
:1042C00015BE00110200000022BE00110300000014
:1042D0005763FF1F0200000018C000110300000018
:1042E0006C63FF1F020000001AC0001101000000F3
:1042F00014BE00110200000020BE001103000000E7
:104300002D63FF1F0200000018C000110300000011
:104310004E63FF1F020000001EC0001101000000DC
:1043200058BE0011020000001AC000110100000078
:10433000E943FF1F020000006ABE001101000000F7
:1043400053BE0011020000001AC00011010000005D
:10435000E843FF1F0200000068BE001101000000DA
:104360007463FF1F020000001AC00011010000006A
:10437000E743FF1F0200000066BE001101000000BD
:1043800043BE0011020000001AC00011010000002D
:10439000E643FF1F0200000064BE001101000000A0
:1043A0003EBE0011020000001AC000110100000012
:1043B000E543FF1F0200000062BE00110100000083
:1043C00039BE0011020000001AC0001101000000F7
:1043D000E443FF1F0200000060BE00110100000066
:1043E00034BE001102020202020200001D4C001144
:1043F000E34B0011ACBE0011900118001800FFFF44
:104400000701020304050602010600000000000087
:10441000000000000000000000000000000000009C
:104420000000000000000300020000001EC0001198
:10443000010000002CBF0011020000001AC0001192
:10444000010000009844FF1F0200000036BF001169
:1044500001000000A263FF1F0200000018C000114D
:10446000030000001066FF1F020000001AC00011C8
:10447000010000009844FF1F0200000034BF00113B
:1044800001000000A463FF1F0200000018C000111B
:10449000030000000866FF1F12A6A6A60000000089
:1044A0000001000000000111FFFF000050485936D4
:1044B000000000000000000001000000BDBE00116F
:1044C0000B000500F7000000B400002800280028B9
:1044D0003075A000A000A000A00000080008E001C6
:1044E000F00010001000100010001000100050002C
:1044F0005000500010001000D00700000000000025
:104500000F0001000500307507001000010081FF59
:1045100000000000FF000000B9740011C17200111A
:1045200051700011FFFF0100FF000000D59E001137
:10453000519C0011699B0011000000000000000068
:1045400000000800040000003B0001085902E001DF
:1045500088212800FF000000020000001EC000119A
:1045600001000000E4C00011020000001AC00011A8
:1045700001000000D545FF1F0200000016C0001119
:1045800001000000246AFF1F020000001AC0001191
:1045900001000000D445FF1F0200000014C00011FC
:1045A00001000000D245FF1F020000001AC00011E8
:1045B00001000000D045FF1F0200000012C00011E2
:1045C00001000000C845FF1F1800180000009001FE
:1045D0000200000302020000020000001EC00011E1
:1045E00001000000F8C00011020000001AC0001114
:1045F000010000001846FF1F0200000010C000115B
:1046000000000000000000000200000018C00011BF
:0A46100003000000446AFF1F20FFB2
:040000051FFF184180
:00000001FF
